:020000020000FC
:040000000C943A48DA
:040038000C94DD5AED
:040050000C94955B1C
:040064000C943D5A61
:04006C000C946C5A2A
:04011C000C94EB470D
:040134000C943B46A6
:04014C000C94CB47FD
:040154000C94BA4706
:1001F00000000000000000000000000000000000FF
:1002000000000000000000000000000000000000EE
:1002100000000000000000000000000000000000DE
:1002200000000000000000000000000000000000CE
:1002300000000000000000000000000000000000BE
:1002400000000000000000000000000000000000AE
:10025000000000000000000000000000000000009E
:10026000000000000000000000000000000000008E
:10027000000000000000000000000000000000007E
:10028000000000000000000000000000000000006E
:10029000000000000000000000000000000000005E
:1002A000000000000000000000000000000000004E
:1002B000000000000000000000000000000000003E
:1002C000000000000000000000000000000000002E
:1002D000000000000000000000000000000000001E
:1002E000000000000000000000000000000000000E
:1002F00000000000000000000000000000000000FE
:1003000000000000000000000000000000000000ED
:1003100000000000000000000000000000000000DD
:1003200000000000000000000000000000000000CD
:1003300000000000000000000000000000000000BD
:1003400000000000000000000000000000000000AD
:10035000000000000000000000000000000000009D
:10036000000000000000000000000000000000008D
:10037000000000000000000000000000000000007D
:10038000000000000000000000000000000000006D
:10039000000000000000000000000000000000005D
:1003A0000000000000000000C060C060E0E0E0E08D
:1003B00071C071C03B803B801F001F000E001F00FA
:1003C0001F003B803B8071C071C0E0E0E0E0C06096
:1003D000000000000000000000000000000000001D
:1003E000000000000000000000000000000000000D
:1003F00000000000000000000000000000000000FD
:1004000000000000000000000000000000000000EC
:1006C0000000000000000000000000000000FFC06B
:1006D000FFC0FFC0000000000000FFC0FFC0FFC05F
:1006E000000000000000FFC0FFC0FFC000000000CD
:1006F00000000000000000000000000000000000FA
:1007000000000000000000000000000000000000E9
:10071000000000000000000000000C001E001E0091
:100720001E001E001E001E001E001E001E001E00D9
:100730000C00000000001E001E001E001E00000035
:10074000F3C0F3C0F3C0F3C0F3C071C06180C30055
:100750008200000000000000000000000000000017
:100760000000000000000000198019801980198025
:100770003300FFC0FFC0FFC0330033006600FFC07E
:10078000FFC0FFC0660066006600CC00CC00000021
:100790000C003F007F80FFC0EDC0EDC0EC00EC001E
:1007A0007C007F003F800FC00DC0EDC0EDC0EDC0EC
:1007B0007F807F803F000C007000F8C0D9C0F9C076
:1007C00073800380070007000E000E001C001C0051
:1007D0003800380070007380E7C0E6C0C7C00380EF
:1007E0001E003F007F807380738073807F803F0096
:1007F0001E003E007C00FEC0F7C0E3C0E380E38043
:10080000F780FFC07FC03CC01E001E001E001E00FF
:100810001E000E000E001C0018000000000000006A
:1008200000000000000000000000000000000000C8
:1008300003000F000E001C001C003C0038003800B4
:100840003800380038003800380038003C001C0000
:100850001C000E000F00030030003C001C000E00C6
:100860000E000F0007000700070007000700070041
:10087000070007000F000E000E001C003C003000B7
:100880000000000000000C001E001E00CCC0FFC0D5
:10089000FFC0DE401F007F80738033000000000037
:1008A0000000000000000000000000001E001E000C
:1008B0001E001E00FFC0FFC0FFC0FFC01E001E00C4
:1008C0001E001E00000000000000000000000000EC
:1008D0000000000000000000000000000000000018
:1008E0000000000000001E001E001E001E001E0072
:1008F0000E000E001C0018000000000000000000A8
:1009000000000000FFC0FFC0FFC0FFC000000000EB
:1009100000000000000000000000000000000000D7
:1009200000000000000000000000000000000000C7
:100930000000000000000000000000001E003F005A
:100940003F003F003F001E00000000C001C001C08A
:1009500003800380070007000E000E001C001C002F
:100960003800380070007000E000E000C0000000B7
:100970001E003F007F807380E1C0E1C0E1C0E1C0A4
:10098000E1C0E1C0E1C0E1C0E1C0E1C0E1C0E1C05F
:1009900073807F803F001E0007000F001F003F0094
:1009A0007F00770067004700070007000700070087
:1009B00007000700070007000700070007000700FF
:1009C0003F007F80FFC0F3C0E1C0E1C001C001C0B3
:1009D00001C0038007800F001E003C007800F0007B
:1009E000E000FFC0FFC0FFC01F003F807FC073C09A
:1009F00061C001C001C003800F000E000F800380A2
:100A000001C001C001C0C1C0E3C0FF807F803E00C3
:100A10000380078007800F801F801F803F807B80BE
:100A20007380E380E380FFC0FFC0FFC003800380CA
:100A300003800380038003803F807F807F8070007D
:100A40007000E000E000EF00FF80FFC0F3C0E1C0F5
:100A500001C001C001C0C1C0E380FF807F003E0033
:100A60001E003F007F807380E180E000E000EE0028
:100A7000FF00FF80F3C0E1C0E1C0E1C0E1C0E1C020
:100A8000F3C07F803F001E00FFC0FFC0FFC001C059
:100A900003800380070007000E000E001C001C00EE
:100AA00038003800700070007000E000E000E000E6
:100AB0001E003F007F807380618061806180738051
:100AC0003F003F007F80F3C0E1C0E1C0E1C0E1C072
:100AD000F3C07F803F001E001E007F807F80F3C038
:100AE000E1C0E1C0E1C0E1C0E1C0F3C07FC07FC0B0
:100AF0003FC001C001C0C1C0E380FF807F003E0055
:100B00000000000000003C003C003C003C000000F5
:100B100000000000000000003C003C003C003C00E5
:100B200000000000000000000000000000003C0089
:100B30003C003C003C000000000000000000000001
:100B40003C003C003C003C000C001C003800000055
:100B5000000000800180038007800F001E003C0021
:100B60007800F000E000F00078003C001E000F006C
:100B7000078003800180008000000000000000006A
:100B80000000FF80FF80FF80000000000000FF8069
:100B9000FF80FF8000000000000000000000000057
:100BA000000040006000700078003C001E000F0054
:100BB000078003C001C003C007800F001E003C0077
:100BC00078007000600040001E003F007F80F380CE
:100BD000E3C0E1C0E1C001C001C003C003800780E1
:100BE0000F001E001C00000000001C001C001C0068
:100BF0003F007F80FFC0E1C0CCC0DEC0DEC0D2C0FD
:100C0000D2C0D2C0D2C0D2C0DEC0DEC0CF80C7004A
:100C1000E040FFC07FC03F800FC01FC01FC01DC08D
:100C20001DC039C039C039C039C039C071C071C0A8
:100C30007FC07FC07FC0FFC0E1C0E1C0E1C0E1C0B4
:100C4000FE00FF00FF80E780E380E380E380E78031
:100C5000FF80FF00FF80E3C0E1C0E1C0E1C0E1C070
:100C6000E3C0FFC0FF80FF001E003F007F807FC009
:100C7000F1C0E0C0E0C0E000E000E000E000E00023
:100C8000E000E0C0E0C0F1C07FC07F803F001E00F8
:100C9000FC00FE00FF00FF80E780E3C0E1C0E1C090
:100CA000E1C0E1C0E1C0E1C0E1C0E3C0E380E780B2
:100CB000FF80FF00FE00FC00FFC0FFC0FFC0FFC0C0
:100CC000E000E000E000E000FF00FF00FF00FF00A8
:100CD000E000E000E000E000FFC0FFC0FFC0FFC098
:100CE000FFC0FFC0FFC0FFC0E000E000E000E00088
:100CF000FF80FF80FF80E000E000E000E000E00017
:100D0000E000E000E000E0001E003F007F807F8008
:100D1000F1C0E1C0E000E000E000E7C0E7C0E7C0EC
:100D2000E7C0E7C0E0C0F1C07FC07F803F801E0009
:100D3000E1C0E1C0E1C0E1C0E1C0E1C0E1C0E1C0AB
:100D4000FFC0FFC0FFC0FFC0E1C0E1C0E1C0E1C023
:100D5000E1C0E1C0E1C0E1C00E000E000E000E00D7
:100D60000E000E000E000E000E000E000E000E0013
:100D70000E000E000E000E000E000E000E000E0003
:100D800001C001C001C001C001C001C001C001C05B
:100D900001C001C001C001C0E1C0E1C0E1C0F3C0B9
:100DA0007FC07FC03F801F00E1C0E1C0E380E380DF
:100DB000E700E700EE00FE00FC00FE00EE00EF00A2
:100DC000E700E780E380E380E3C0E1C0E1C0E1C089
:100DD000E000E000E000E000E000E000E000E00013
:100DE000E000E000E000E000E000E000E000E00003
:100DF000FFC0FFC0FFC0FFC0C0C0E1C0E1C0E1C094
:100E0000F3C0F3C0FFC0FFC0FFC0FFC0EDC0EDC026
:100E1000EDC0EDC0EDC0E1C0E1C0E1C0E1C0E1C0A6
:100E2000E1C0E1C0E1C0F1C0F1C0F9C0F9C0F9C052
:100E3000FDC0EDC0EDC0EFC0E7C0E7C0E7C0E3C054
:100E4000E3C0E1C0E1C0E1C01E003F007F807F80C1
:100E5000F3C0E1C0E1C0E1C0E1C0E1C0E1C0E1C078
:100E6000E1C0E1C0E1C0F3C07F807F803F001E0091
:100E7000FC00FF00FF80FFC0E3C0E1C0E1C0E3C0B1
:100E8000FFC0FF80FF00FC00E000E000E000E000A9
:100E9000E000E000E000E0003C007E007F00FF009A
:100EA000F780E380E380E380E380E380E380E38016
:100EB000EB80EF80EF80EF007F007F803DC019C0A6
:100EC000FC00FF00FF80FFC0E3C0E1C0E1C0E3C061
:100ED000FF80FF00FE00FF00E700E780E380E38083
:100EE000E3C0E1C0E1C0E1C01E003F003F807FC021
:100EF0007BC071C071C078007C003F001F800FC0B4
:100F000003C0E1C0E1C0F3C07FC07F803F801E000E
:100F1000FFC0FFC0FFC0FFC01E001E001E001E005D
:100F20001E001E001E001E001E001E001E001E00D1
:100F30001E001E001E001E00E1C0E1C0E1C0E1C0B5
:100F4000E1C0E1C0E1C0E1C0E1C0E1C0E1C0E1C099
:100F5000E1C0E1C0E1C0F3C07F807F803F001E00A0
:100F6000E1C0E1C0E1C0E1C0E180618061807380E7
:100F70007380738073803300330033003F001E00A2
:100F80001E001E000C000C00E1C0E1C0E1C0E1C089
:100F9000E1C0EDC0EDC0EDC0EDC0EDC0EDC0EDC0F5
:100FA000EDC0FFC0FFC07F8073807380618061806F
:100FB000E1C0E1C0E1C0E1C07380738073803F0095
:100FC0001E001E001E003F007F8073807380E1C002
:100FD000E1C0E1C0E1C0E1C0E1C0E1C0E1C0E1C009
:100FE0007380738073003F001E001E000C000C0015
:100FF0000C000C000C000C000C000C000C000C0091
:101000003FC03FC03FC03FC001C003800380070016
:1010100007000E000E001C001C0038003800700095
:101020007FC07FC07FC07FC0000000001F001F0086
:101030001F001C001C001C001C001C001C001C00CD
:101040001C001C001C001C001C001F001F001F00B7
:101050000000000070007000700038003800380098
:10106000380038001C001C001C001C001C000E0076
:101070000E000E0000000000000000001F001F0016
:101080001F00070007000700070007000700070010
:10109000070007000700070007001F001F001F00D0
:1010A00008001C003E003E0077007700E380E380EC
:1010B0000000000000000000000000000000000030
:1010C0000000000000000000000000000000000020
:1010D0000000000000000000000000000000000010
:1010E00000000000000000000000FFC0FFC0FFC0C3
:1010F00000001E000E0007000300000000000000BA
:1011000000000000000000000000000000000000DF
:1011100000000000000000000000000000000000CF
:1011200000003E007F00FF80C78003801F807F801B
:10113000FF80E780C380C380E780FF807FC039C025
:10114000E000E000E000E000E000EF00FF80FF8052
:10115000F3C0E1C0E1C0E1C0E1C0E1C0E1C0E1C075
:10116000F3C0FF80FF80EF000000000000000000DF
:1011700000003F007F80FF80F3C0E1C0E000E0009E
:10118000E000E000E000E1C0F3C0FF807F803F00AE
:1011900001C001C001C001C001C03DC07FC07FC00F
:1011A000F3C0E1C0E1C0E1C0E1C0E1C0E1C0E1C025
:1011B000F3C07FC07FC03DC0000000000000000001
:1011C00000003F007F807F80F3C0E1C0FFC0FFC010
:1011D000FFC0E000E000E1C0F3C07F807F803F00FF
:1011E0000F801F801F801C001C007F007F007F007D
:1011F0007F001C001C001C001C001C001C001C00AC
:101200001C001C001C001C0000000000000000006E
:101210003DC07FC0FFC0F3C0E1C0E1C0E1C0E1C09C
:10122000F3C0FFC07FC03FC001C0E3C0FFC07F80EC
:101230007000700070007000700077007F807FC0C9
:101240007BC071C071C071C071C071C071C071C00C
:1012500071C071C071C071C01C001C001C00000076
:1012600000001C001C001C001C001C001C001C00BA
:101270001C001C001C001C001C001C001C001C008E
:101280001C001C001C00000000001C001C001C00B6
:101290001C001C001C001C001C001C001C001C006E
:1012A0001C007C007C007800E000E000E000E00032
:1012B000E000E1C0E3C0E780E700EE00FC00FC00D6
:1012C000FE00EE00E700E700E380E3C0E1C0E1C01C
:1012D0001C001C001C001C001C001C001C001C002E
:1012E0001C001C001C001C001C001C001C001C001E
:1012F0001C001C001C001C0000000000000000007E
:101300000000DB80FFC0FFC0FFC0DDC0CCC0CCC090
:10131000CCC0CCC0CCC0CCC0CCC0CCC0CCC0CCC06D
:1013200000000000000000000000EE00FF80FFC091
:10133000FFC0F3C0E1C0E1C0E1C0E1C0E1C0E1C075
:10134000E1C0E1C0E1C0E1C0000000000000000019
:1013500000003F007F80FFC0F3C0E1C0E1C0E1C0FA
:10136000E1C0E1C0E1C0E1C0F3C0FFC07F803F0049
:10137000000000000000EF00FF80FFC0FBC0F1C0D4
:10138000F1C0F1C0F1C0FBC0FFC0FF80EF00E00082
:10139000E000E000E000E0000000000000000000CD
:1013A00000001DC07FC07FC0F3C0E1C0E1C0E1C04C
:1013B000E1C0F3C07FC07FC01FC001C001C001C039
:1013C00000000000000000000000E3C0FFC0FFC0FC
:1013D000F800F000E000E000E000E000E000E000E5
:1013E000E000E000E000E00000000000000000007D
:1013F00000003F007F80FFC0F1C0E000F0007C00F3
:101400003F800FC003C001C0E3C0FFC07F803F002A
:10141000000004000C001C001C003F003F003F00C7
:101420001C001C001C001C001C001C001C001C00DC
:101430001C001F001F000F00000000000000000043
:101440000000E1C0E1C0E1C0E1C0E1C0E1C0E1C035
:10145000E1C0E1C0E1C0E1C0F3C0FFC07FC03DC05A
:1014600000000000000000000000E1C0E1C0E1C099
:10147000E1C0E1C0F3C07380738073803F003F0020
:101480001E001E000C000C00000000000000000008
:101490000000C0C0C0C0CCC0CCC0EDC0EDC0EDC02D
:1014A0006D806D807F807F807F803F0033003300C0
:1014B00000000000000000000000E1C0E1C0E1C049
:1014C00073803F001E001E001E001E003F007F8034
:1014D000F3C0E1C0E1C0E1C0000000000000000076
:1014E0000000E1C0E1C071C071C071C03B803B80B1
:1014F0003B001F001F000E001E007C007C007800D7
:1015000000000000000000000000FFC0FFC0FFC09E
:1015100003C0078007800F001E001C003C007800FD
:10152000F000FFC0FFC0FFC007000F001F001C003D
:101530001C001C001C001C003C00780078003C00D3
:101540001C001C001C001C001C001F000F000700DA
:101550001C001C001C001C001C001C001C001C00AB
:101560001C001C001C001C001C001C001C001C009B
:101570001C001C001C001C00700078007C001C007B
:101580001C001C001C001C001E000F000F001E0091
:101590001C001C001C001C001C007C00780070005B
:1015A00000000000000078C0FDC0EFC0C780000050
:1015B000000000000000000000000000000000002B
:1015C000000000000000000000000000000000001B
:1015D000000000000000000000000000000000000B
:1015E00000000000000000000000000000000000FB
:1015F000FF00FF00FF0070007000700070007000BE
:101600007E007F007F80738073807380738073801F
:1016100073807780770076000F003F003C00000069
:10162000FF80FF80FF80E000E000E000E000E000DD
:10163000E000E000E000E000E000E000E000E000AA
:10164000000000000000000000000000000000009A
:101650000000000000000000000000003C003C0012
:101660003C000C000C001800000000000F003F00C0
:101670003C000000FF80FF80FF80E000E000E00011
:10168000E000E000E000E000E000E000E000E0005A
:10169000000000000000000000000000000000004A
:1016A000000000000000000000000000F3C0F3C0D4
:1016B000F3C030C030C061800000000000000000B6
:1016C000000000000000000000000000000000001A
:1016D00000000000000000000000EEE0EEE0EEE0A0
:1016E0000000000000001C001C001C001C00FF800B
:1016F000FF80FF801C001C001C001C001C001C0044
:101700001C001C001C001C000000000000001C004D
:101710001C001C001C00FF80FF80FF801C001C00C0
:101720001C00FF80FF80FF801C001C001C001C00B0
:10173000000000001F003F807FC0F1C0E0C0E0005B
:10174000FF00FF00E000E000FF00FF00E000E0001D
:10175000F1C07FC03F801F000000000000000000BB
:101760007000704050C071C073C007800F001E0031
:101770003C00780070006EE04EE00AA00EE00EE043
:101780001F003F007F007700770077007700770029
:10179000778077C077E077E0776077607760776011
:1017A00077E0F7E0E7C0C7800000000000000040DD
:1017B00000C001C0038007000E001C00380070004C
:1017C00038001C000E000700038001C000C000406C
:1017D000EE00EE00EE00EE00EE00EE00EE00EE0099
:1017E000FF00FF80EFC0EFC0EEC0EEC0EEC0EEC065
:1017F000EFC0EFC0EF80EF000F003F003C000000A3
:10180000E180E380E700EE00FC00F800F000E0007B
:10181000F000F800FC00EE00E700E380E1C0E0C06B
:10182000FF80FF80FF8038003800380038003F001C
:101830003F803FC039C039C039C039C039C039C014
:1018400039C039C039C039C0E1C0E1C0E1C0E1C030
:10185000E1C0E1C0E1C0E1C0FFC0FFC07F801E0069
:101860001E001E001E001E001E001E001E001E0088
:101870000000000038003800FF80FF80FF80380043
:10188000380038003F003F803BC039C039C039C004
:1018900039C03BC03F803F000C00180018001E00FC
:1018A0001E001E00000000000000000000000000FC
:1018B0000000000000000000000000000000000028
:1018C0001E001E001E00060006000C0000000000A6
:1018D0000000000000000000000000000000000008
:1018E00000000000000000006180C300C300F3C0DE
:1018F000F3C0F3C000000000000000000000000082
:1019000000000000000000000000000000000000D7
:10191000F3C0F3C0F3C030C030C0618000000000ED
:1019200000000000000000000000000000000000B7
:1019300000000000000000000000000000000000A7
:1019400000000000000000001E003F003F003F00BC
:101950003F001E000000000000000000000000002A
:101960000000000000000000000000000000000077
:10197000000000003E003E003E00000000000000AD
:101980000000000000000000000000000000000057
:10199000000000000000000000000000FFC0FFC0C9
:1019A000FFC0000000000000000000000000000078
:1019B0000000000000000000000000000000000027
:1019C0000000000000000000000000000000000017
:1019D00000000000000000000000FC4026C027C0FE
:1019E00025402440244000000000000000000000CA
:1019F00000000000000000000000000000000000E7
:101A0000000000000000000000001F003F007F00F9
:101A100077007700778077C077E0776077607760CE
:101A20007760F7E0E7C0C78000000000000080009A
:101A3000C000E000700038001C000E0007000380AA
:101A400007000E001C0038007000E000C00080009D
:101A500000000000000000000000EE00EE00EE00BC
:101A6000EE00EE00FF00FF80FFC0EFC0EEC0EEC052
:101A7000EFC0EFC0EF80EF00000000001E007E000E
:101A800078000000E380E700EE00FC00F800F000C2
:101A9000E000F000F800FC00EE00E700E380E1C0A9
:101AA0000000000070007000F800F800F8007000FE
:101AB000700077007F807FC07BC071C071C071C033
:101AC00071C071C071C071C0000000000000000052
:101AD0000000E1C0E1C0E1C0E1C0E1C0E1C0E1C09F
:101AE000E1C0FFC0FFC07F801E001E001E001E0060
:101AF00000000000000000000000000000000000E6
:101B000000000000000000000000000000000000D5
:101B1000000000000000000061807F801E00E1C026
:101B2000E1C0E1C0E1C0E1C0E1C0F3C073807F80EB
:101B30003F003F001E001E003E00FC00F800F000C9
:101B400000000000000061807F801E00E1C0E1C055
:101B5000E1C0E1C073807F803F003F001E001E0097
:101B60003E00FC00F800F000038003800380038047
:101B7000038003800380038003800380038003804D
:101B8000038003800380E380F780FF807F003E00B6
:101B9000000000000000000000000000C0C0EDC018
:101BA0007F8033006180618033007F80EDC0C0C0E2
:101BB000000000000000000001C001C0FFC0FFC025
:101BC000FFC0E000E000E000E000E000E000E00036
:101BD000E000E000E000E000E000E000E000E00005
:101BE00000000000380038003800380038003800A5
:101BF0003800380000000000380038003800380095
:101C000038003800380038003E007F00FF80E38055
:101C1000E180F0007E007F00FF80E380E380FF80B2
:101C20007F003F000780C380E380FF807F003E008D
:101C3000330033000000FF80FF80FF80E080E00081
:101C4000E000FE00FE00FE00E000E000E000E0003A
:101C5000E000FF80FF80FF80000000000000000027
:101C60003F807FC0FFE0E0E0CE60DF60DB60D860F7
:101C7000DB60DF60CE60E0E0FFE07FC03F8000001F
:101C80001F003F807FC0F1C0E000E000E000FF00E7
:101C9000FF00FF00E000E000E000E000E000E00006
:101CA000F1C07FC03F801F00000000000000000066
:101CB000000000000000084018C039C07380E70031
:101CC000738039C018C00840000000000000000008
:101CD0000000000000000000000000000000000004
:101CE000000000000000000000000000FFC0FFC076
:101CF000FFC001C001C000000000000000000000A3
:101D000000000000000000007F807F807F800000D6
:101D100000000000000000000000000000000000C3
:101D2000000000003F807FC0FFE0E0E0C060DE60B8
:101D3000DF60DB60DB60DF60DE60DF60DB60C060D7
:101D4000E0E0FFE07FC03F801B001B0000000E00B2
:101D50000E000E000E000E000E000E000E000E0013
:101D60000E000E000E000E000E000E000E000E0003
:101D700000001B003B003B8071C071C03B801B001A
:101D80001B00000000000000000000000000000038
:101D90000000000000000000000000000000000043
:101DA0000E000E000E007FC07FC07FC00E000E0030
:101DB0000E0000007FC07FC07FC000000000000058
:101DC0000E000E000E000E000E000E000E000E00A3
:101DD0000E000E000E000E000E000E000E000E0093
:101DE0000E000E000E000E0000001C001C001C0067
:101DF00000001C001C001C001C001C001C001C001F
:101E00001C001C001C001C001C001C001C001C00F2
:101E100000000000000001C001C0FFC0FFC0FFC003
:101E2000E000E000E000E000E000E000E000E000B2
:101E3000E000E000E000E000000000000000000022
:101E40000000E380E380E380E380E380E380E380DD
:101E5000F780FF80FF80EB80E000E000E000E00022
:101E6000000000003FC07FC0FFC0FDC0FDC0FDC03E
:101E7000FDC0FDC07DC03DC01DC01DC01DC01DC03A
:101E80001DC01DC01DC01DC00000000000000000DE
:101E900000000000000000001E001E001E001E00CA
:101EA0000000000000000000000000000000000032
:101EB000000033003300000000003F007F80FFC0BF
:101EC000F3C0E1C0E1C0FFC0FFC0FF80E000E00060
:101ED000F1C0FFC07F803F00C600C600C600C6003C
:101EE000C600E600E600F680FFC0DFC0CF40CF406E
:101EF000C740C7C0C7C0C680C600C7C0C7C0C7C02C
:101F0000000000000000000000003F007F80FFC0D4
:101F1000F1C0E000E000FE00FE00FE00E000E00096
:101F2000F1C0FFC07F803F00000000000000000003
:101F3000000000000000000000008400C600E70070
:101F4000738039C07380E700C60084000000000081
:101F500001C001C001C0000001C001C001C001C03A
:101F600001C001C001C001C001C001C001C071C0F9
:101F70007BC07FC03F801F001E003F007F80F3803A
:101F8000E000E000E000F0007E003F001F8003C0A2
:101F900001C000C001C0C1C0E3C0FF807F003E009F
:101FA000000000000000000000003F007F80FFC034
:101FB000F1C0E000F000FF007F803FC003C0C1C05F
:101FC000E3C0FFC07F803F00000000001B001B003B
:101FD000000000000E000E000E000E000E000E00AD
:101FE0000E000E000E000E000E000E000E000E0081
:101FF0000FC01FC01FC01DC01DC039C039C039C0AF
:1020000039C039C071C071C07FC07FC07FC0FFC000
:10201000E1C0E1C0E1C0E1C0FF80FF80FF80E000DF
:10202000E000E000E000FE00FF00FF80FFC0E3C032
:10203000E1C0E1C0E1C0E3C0FFC0FF80FF80FE005F
:10204000FE00FF00FF80E780E380E380E380E7801D
:10205000FF80FF00FF80E3C0E1C0E1C0E1C0E1C05C
:10206000E3C0FFC0FF80FF00FFC0FFC0FFC0FFC094
:10207000E000E000E000E000E000E000E000E00060
:10208000E000E000E000E000E000E000E000E00050
:102090003F803F803F803B803B803B803B803B805C
:1020A0007B80738073807380738073807380FFC0C4
:1020B000FFC0FFC0E1C0E1C0FFC0FFC0FFC0FFC064
:1020C000E000E000E000E000FF00FF00FF00FF0094
:1020D000E000E000E000E000FFC0FFC0FFC0FFC084
:1020E000EDC0EDC0EDC0EDC0EDC06D806D803F0076
:1020F0001E003F007F806D806D80EDC0EDC0EDC0A3
:10210000EDC0EDC0EDC0EDC03E007F00FF00FF80E0
:10211000E780C380438007801F001F800F8001C0BD
:1021200001C0C1C0C1C0E3C0FFC0FFC07F801E00AE
:10213000E1C0E1C0E1C0E1C0E3C0E3C0E7C0E7C087
:10214000EFC0EFC0FDC0F9C0F9C0F1C0F1C0E1C0FF
:10215000E1C0E1C0E1C0E1C0DEC0DEC0CCC0C0C0B3
:10216000E1C0E1C0E3C0E7C0E7C0EFC0FDC0F9C017
:10217000F9C0F1C0F1C0E1C0E1C0E1C0E1C0E1C01F
:10218000E1C0E1C0E380E380E700E700EE00FE008D
:10219000FC00FE00EE00EF00E700E780E380E38054
:1021A000E3C0E1C0E1C0E1C03FC03FC03FC03FC0AD
:1021B00039C039C039C039C039C039C039C039C057
:1021C00039C039C039C039C039C0F9C0F1C0E1C027
:1021D000C0C0E1C0E1C0E1C0F3C0F3C0FFC0FFC0B8
:1021E000FFC0FFC0EDC0EDC0EDC0EDC0EDC0E1C06F
:1021F000E1C0E1C0E1C0E1C0E1C0E1C0E1C0E1C0D7
:10220000E1C0E1C0E1C0E1C0FFC0FFC0FFC0FFC04E
:10221000E1C0E1C0E1C0E1C0E1C0E1C0E1C0E1C0B6
:102220001E003F007F807F80F3C0E1C0E1C0E1C0BD
:10223000E1C0E1C0E1C0E1C0E1C0E1C0E1C0F3C084
:102240007F807F803F001E00FFC0FFC0FFC0FFC037
:10225000E1C0E1C0E1C0E1C0E1C0E1C0E1C0E1C076
:10226000E1C0E1C0E1C0E1C0E1C0E1C0E1C0E1C066
:10227000FC00FF00FF80FFC0E3C0E1C0E1C0E3C09D
:10228000FFC0FF80FF00FC00E000E000E000E00095
:10229000E000E000E000E0001E003F007F807FC023
:1022A000F1C0E0C0E0C0E000E000E000E000E000DD
:1022B000E000E0C0E0C0F1C07FC07F803F001E00B2
:1022C000FFC0FFC0FFC0FFC01E001E001E001E009A
:1022D0001E001E001E001E001E001E001E001E000E
:1022E0001E001E001E001E00E1C0E1C0E1C0E1C0F2
:1022F000E1C0E1C0738073803F003F001F001F00FA
:102300000E000E000E000E000E00FC00FC00F80097
:102310001E001E003F007F80FFC0FFC0EDC0CCC08C
:10232000CCC0CCC0CCC0CCC0EDC0FFC0FFC07F8053
:102330003F001E001E001E00E1C0E1C0E1C0E1C080
:102340007380738073803F001E001E001E003F00DC
:102350007F8073807380E1C0E1C0E1C0E1C0E1C073
:10236000E380E380E380E380E380E380E380E38055
:10237000E380E380E380E380E380E380E3C0FFC0A9
:10238000FFC0FFC001C001C0E1C0E1C0E1C0E1C0C9
:10239000E1C0E1C0E1C0E1C0F1C0FFC0FFC07FC04B
:1023A0003FC001C001C001C001C001C001C001C0E7
:1023B000CCC0CCC0CCC0CCC0CCC0CCC0CCC0CCC0BD
:1023C000CCC0CCC0CCC0CCC0CCC0CCC0CCC0CCC0AD
:1023D000FFC0FFC0FFC0FFC0CCC0CCC0CCC0CCC0D1
:1023E000CCC0CCC0CCC0CCC0CCC0CCC0CCC0CCC08D
:1023F000CCC0CCC0FFC0FFC0FFC0FFC000C000C049
:10240000F000F000F000F00030003000300030004C
:102410003E003F803FC03FC031C030C030C031C0FF
:102420003FC03FC03F803E00C0C0C0C0C0C0C0C0B1
:10243000C0C0C0C0C0C0C0C0C0C0F8C0FCC0FEC0EA
:10244000CEC0C6C0C6C0C6C0CEC0FEC0FCC0F8C0AC
:10245000E000E000E000E000E000E000E000E0007C
:10246000FE00FF00FF80FF80E3C0E1C0E1C0E3C0E9
:10247000FF80FF80FF00FE003E007F007F80FF8026
:10248000F3C0E1C0C1C001C00FC01FC01FC00FC05A
:1024900001C0C1C0E1C0F3C0FF807F807F003E006B
:1024A000C700CF80DFC0DFC0DDC0D8C0D8C0F8C053
:1024B000F8C0F8C0F8C0F8C0F8C0D8C0D8C0DDC0B7
:1024C000DFC0DFC0CF80C7000FC03FC07FC0FFC0EC
:1024D000F1C0E1C0E1C0F1C07FC03FC01FC03FC03C
:1024E00039C039C079C079C0F1C0F1C0E1C0E1C0E4
:1024F000000000000000000000003E007F00FF80A0
:10250000C78003801F807F80FF80E780C380C380F7
:10251000E780FF807FC039C000001FC07FC0FFC0C0
:10252000E000C000DF00FF80FFC0F3C0E1C0E1C0F9
:10253000E1C0E1C0E1C0E1C0F3C0FFC07F803F0067
:1025400000000000000000000000FE00FF00FF800F
:10255000E780E380E700FE00FF00FF80E3C0E1C00A
:10256000E3C0FFC0FF80FF0000000000000000008B
:102570000000FFC0FFC0FFC0F000F000F000F0005E
:10258000F000F000F000F000F000F000F000F000CB
:10259000000000000000000000003F803F803F80FE
:1025A0003B803B803B807380738073807380FFC06F
:1025B000FFC0FFC0E1C0E1C000000000000000005B
:1025C00000003F007F807F80F3C0E1C0FFC0FFC0FC
:1025D000FFC0E000E000E1C0F3C07F807F803F00EB
:1025E00000000000000000000000EDC0EDC0EDC0E4
:1025F0006D807F807F803F003F006D806D806D80AB
:10260000EDC0EDC0EDC0EDC0000000000000000016
:1026100000007F00FF80FFC063C001C0078007008B
:10262000078003C001C001C063C0FFC0FF807F00FE
:1026300000000000000000000000E1C0E1C0E3C0B5
:10264000E3C0E7C0E7C0EFC0EDC0FDC0F9C0F9C00E
:10265000F1C0F1C0E1C0E1C033003F003F001E0007
:102660000000E1C0E1C0E3C0E3C0E7C0E7C0EFC0E5
:10267000EDC0FDC0F9C0F9C0F1C0F1C0E1C0E1C0DA
:1026800000000000000000000000E1C0E3C0E7809F
:10269000E700EE00FC00FC00FE00EE00E700E700B3
:1026A000E380E3C0E1C0E1C00000000000000000E2
:1026B00000003FC03FC03FC039C039C039C039C039
:1026C00039C039C039C039C039C0F1C0F1C0E1C02A
:1026D00000000000000000000000E1C0E1C0E1C017
:1026E000E1C0F3C0F3C0F3C0FFC0FFC0EDC0EDC058
:1026F000EDC0E1C0E1C0E1C000000000000000004A
:102700000000E1C0E1C0E1C0E1C0E1C0FFC0FFC026
:10271000FFC0E1C0E1C0E1C0E1C0E1C0E1C0E1C093
:10272000000000000000000000003F007F80FFC0AC
:10273000F3C0E1C0E1C0E1C0E1C0E1C0E1C0E1C07F
:10274000F3C0FFC07F803F000000000000000000D9
:102750000000FFC0FFC0FFC0E1C0E1C0E1C0E1C0B8
:10276000E1C0E1C0E1C0E1C0E1C0E1C0E1C0E1C061
:1027700000000000000000000000EF00FF80FBC030
:10278000F1C0F1C0F1C0F1C0F1C0FBC0FF80EF00AB
:10279000E000E000E000E0000000000000000000B9
:1027A00000003F007F80FF80F3C0E1C0E000E00058
:1027B000E000E000E000E1C0F3C0FF807F803F0068
:1027C00000000000000000000000FFC0FFC0FFC0CC
:1027D0001E001E001E001E001E001E001E001E0009
:1027E0001E001E001E001E00000000000000000071
:1027F0000000E1C0E1C071C071C071803B803B80CE
:102800001B001F001F000E001E007C007C007800D3
:1028100000000C000C000C000C006D80FFC0FFC01D
:10282000DEC0CCC0CCC0CCC0DEC0FFC0FFC06D805D
:102830000C000C000C000C00000000000000000068
:10284000000071C071C071C03B801F001F000E00EE
:102850000E000E001F003F807BC071C071C071C0B0
:1028600000000000000000000000E380E380E3803F
:10287000E380E380E380E380E380E380E380FFC0E4
:10288000FFC0FFC003C003C0000000000000000044
:102890000000E1C0E1C0E1C0E1C0E1C0E1C0F1C0C1
:1028A000FFC07FC03FC001C001C001C001C001C066
:1028B00000000000000000000000CCC0CCC0CCC074
:1028C000CCC0CCC0CCC0CCC0CCC0CCC0CCC0CCC0A8
:1028D000CCC0FFC0FFC0FFC000000000000000002F
:1028E0000000CCC0CCC0CCC0CCC0CCC0CCC0CCC014
:1028F000CCC0CCC0CCC0FFC0FFC0FFC000C000C077
:1029000000000000000000000000F800F800F800DF
:102910003800380038003F003F803FC039C038C021
:1029200039C03FC03FC03F800000000000000000F1
:102930000000C0C0C0C0C0C0C0C0C0C0FCC0FEC09D
:10294000FEC0CEC0C6C0C6C0CEC0FEC0FCC0F8C06F
:1029500000000000000000000000E000E000E000D7
:10296000E000E000FF00FF80FFC0E3C0E1C0E1C085
:10297000E3C0FFC0FF80FF00000000000000000077
:1029800000007F00FF80FFC063C001C001C00FC016
:102990000FC00FC001C001C063C0FFC0FF807F0037
:1029A00000000000000000000000C700CF80DFC072
:1029B000DDC0D8C0F8C0F8C0F8C0D8C0D8C0D8C0F2
:1029C000DDC0DF80CF80C7000000000000000000F5
:1029D00000001FC03FC07FC079C071C071C079C006
:1029E0003FC01FC03FC039C079C071C0F1C0E1C055
:1029F000F0011802400268029002B802E0020803E7
:102A0000300358038003A803D003F80320044804CC
:102A100070049804C004E8041005380560058805B2
:102A2000B005D8050006280650067806A006C80698
:102A3000F0061807400768079007B807E00708087E
:102A4000300858088008A808D008F8082009480964
:102A500070099809C009E809100A380A600A880A4A
:102A6000B00AD80A000B280B500B780BA00BC80B30
:102A7000F00B180C400C680C900CB80CE00C080D16
:102A8000300D580D800DA80DD00DF80D200E480EFC
:102A9000700E980EC00EE80E100F380F600F880FE2
:102AA000B00FD80F0010281050107810A010C810C8
:102AB000F0101811401168119011B811E0110812AE
:102AC000301258128012A812D012F8122013481394
:102AD00070139813C013E81310143814601488147A
:102AE000B014D8140015281550157815A015C81560
:102AF000F0151816401668169016B816E016081746
:102B0000301758178017A817D017F817201848182B
:102B100070189818C018E818101938196019881911
:102B2000B019D819001A281A501A781AA01AC81AF7
:102B3000F01A181B401B681B901BB81BE01B081CDD
:102B4000301C581C801CA81CD01CF81C201D481DC3
:102B5000701D981DC01DE81D101E381E601E881EA9
:102B6000B01ED81E001F281F501F781FA01FC81F8F
:102B7000F01F1820402068209020B820E020082175
:102B8000302158218021A821D021F821202248225B
:102B900070229822C022E822102338236023882341
:102BA000B023D8230024282450247824A024C82427
:102BB000F0241825402568259025B825E02508260D
:102BC000302658268026A826D026F82620274827F3
:102BD00070279827C027E8271028382860288828D9
:102BE000B028D8280029282950297829A029C829BF
:102BF00000000000000000000000000000000000D5
:102C000000000000000000000000000000000000C4
:102C100000000000000000000000000000000000B4
:102C200000000000000000000000000000000000A4
:102C30000000000000000000000000000000000094
:102C40000000000000000000000000000000000084
:102C50000000000000000000000000000000000074
:102C60000000000000000000000000000000000064
:102C70000000000000000000000000000000000054
:102C80000000000000000000000000000000000044
:102C90000000000000000000000000000000000034
:102CA0000000000000000000000000000000000024
:102CB0000000000000000000000000000000000014
:102CC0000000000000000000000000000000000004
:102CD00000000000000000000000000000000000F4
:102CE00000000000000000000000000000000000E4
:102CF00000000000000000000000000000000000D4
:102D000000000000000000000000000000000000C3
:102D100000000000000000000000000000000000B3
:102D200000000000000000000000000000000000A3
:102D30000000000000000000000000000000000093
:102D40000000000000000000000000000000000083
:102D50000000000000000000000000000000000073
:102D60000000000000000000000000000000000063
:102D70000000000000000000000000000000000053
:102D80000000000000000000000000000000000043
:102D90000000000000000000000000000000000033
:102DA0000000000000000000C060C060E0E0E0E063
:102DB00071C071C03B803B801F001F000E001F00D0
:102DC0001F003B803B8071C071C0E0E0E0E0C0606C
:102DD00000000000000000000000000000000000F3
:102DE00000000000000000000000000000000000E3
:102DF00000000000000000000000000000000000D3
:102E000000000000000000000000000000000000C2
:1030C0000000000000000000000000000000FFC041
:1030D000FFC0FFC0000000000000FFC0FFC0FFC035
:1030E000000000000000FFC0FFC0FFC000000000A3
:1030F00000000000000000000000000000000000D0
:1031000000000000000000000000000000000000BF
:10311000000000000000000000000C001E001E0067
:103120001E001E001E001E001E001E001E001E00AF
:103130000C00000000001E001E001E001E0000000B
:10314000F3C0F3C0F3C0F3C0F3C071C06180C3002B
:1031500082000000000000000000000000000000ED
:1031600000000000000000001980198019801980FB
:103170003300FFC0FFC0FFC0330033006600FFC054
:10318000FFC0FFC0660066006600CC00CC000000F7
:103190000C003F007F80FFC0EDC0EDC0EC00EC00F4
:1031A0007C007F003F800FC00DC0EDC0EDC0EDC0C2
:1031B0007F807F803F000C007000F8C0D9C0F9C04C
:1031C00073800380070007000E000E001C001C0027
:1031D0003800380070007380E7C0E6C0C7C00380C5
:1031E0001E003F007F807380738073807F803F006C
:1031F0001E003E007C00FEC0F7C0E3C0E380E38019
:10320000F780FFC07FC03CC01E001E001E001E00D5
:103210001E000E000E001C00180000000000000040
:10322000000000000000000000000000000000009E
:1032300003000F000E001C001C003C00380038008A
:103240003800380038003800380038003C001C00D6
:103250001C000E000F00030030003C001C000E009C
:103260000E000F0007000700070007000700070017
:10327000070007000F000E000E001C003C0030008D
:103280000000000000000C001E001E00CCC0FFC0AB
:10329000FFC0DE401F007F8073803300000000000D
:1032A0000000000000000000000000001E001E00E2
:1032B0001E001E00FFC0FFC0FFC0FFC01E001E009A
:1032C0001E001E00000000000000000000000000C2
:1032D00000000000000000000000000000000000EE
:1032E0000000000000001E001E001E001E001E0048
:1032F0000E000E001C00180000000000000000007E
:1033000000000000FFC0FFC0FFC0FFC000000000C1
:1033100000000000000000000000000000000000AD
:10332000000000000000000000000000000000009D
:103330000000000000000000000000001E003F0030
:103340003F003F003F001E00000000C001C001C060
:1033500003800380070007000E000E001C001C0005
:103360003800380070007000E000E000C00000008D
:1033700007001F801F8039C039C071C071C071C083
:10338000F1C0E1C0E1C0E3C0E380E380E380E70097
:10339000E7007E007E0038000180038003800F80FC
:1033A0001F003F003F0077004700070007000E00A6
:1033B0000E000E000E000E000E001C001C001C0073
:1033C0000F003F803F8079C071C001C001C003C0C1
:1033D00007800F000F001E003C003C003C007800FE
:1033E000F000FF80FF80FF000F001F801F803DC0A6
:1033F00039C001C001C003C00F800F000F0007805B
:10340000038003800380E380F7007E007E003C00A1
:1034100000C001C001C003C007800F800F801F8063
:103420001F803B8073807700E700FFC0FFC0FFC0B4
:1034300007000E000E000E001FC01FC01FC0380086
:103440003800380038003F007F8073C073C001C06F
:1034500001C0E1C0E1C0E380F7807F007F003C0055
:103460000F001F801F8039C079C0700070007E007F
:10347000FF00F780F780E380E380E380E380E38070
:1034800077007E007E003C007FC0FFC0FFC001C00F
:1034900003800700070006000E000C000C001C0053
:1034A0001C003800380038003800700070007000D0
:1034B0000F003F803F807BC071C071C071C07380BE
:1034C0003F003F003F007380E380E380E380E380C0
:1034D000E7007E007E003C000F001F801F803B80C5
:1034E00071C071C071C071C071C07BC07BC03FC072
:1034F0001F8003800380E780E7007E007E003C00A1
:103500000000000000003C003C003C003C000000CB
:1035100000000000000000003C003C003C003C00BB
:1035200000000000000000000000000000003C005F
:103530003C003C003C0000000000000000000000D7
:103540003C003C003C003C000C001C00380000002B
:10355000000000800180038007800F001E003C00F7
:103560007800F000E000F00078003C001E000F0042
:103570000780038001800080000000000000000040
:103580000000FF80FF80FF80000000000000FF803F
:10359000FF80FF800000000000000000000000002D
:1035A000000040006000700078003C001E000F002A
:1035B000078003C001C003C007800F001E003C004D
:1035C00078007000600040001E003F007F80F380A4
:1035D000E3C0E1C0E1C001C001C003C003800780B7
:1035E0000F001E001C00000000001C001C001C003E
:1035F0003F007F80FFC0E1C0CCC0DEC0DEC0D2C0D3
:10360000D2C0D2C0D2C0D2C0DEC0DEC0CF80C70020
:10361000E040FFC07FC03F800380078007800780B5
:103620000F800F800F801D801D801D8039803980A4
:103630007F807FC07FC0E1C0E1C0E1C0C1C0C1C028
:103640003F803FC03FC039C071C071C073C07F8030
:103650007F807F807F8071C071C071C0E1C0E1C098
:10366000E3C0FF80FF80FF000F003F803F807BC0F2
:1036700071C071C0F000E000E000E000E000E00098
:10368000E000E000E380E380F7007F007F003C0083
:103690003F003F803F803BC071C071C071C071C0AE
:1036A00071C071C071C073C073807380E380E380A8
:1036B000E780FF00FF00FC003F803F803F80380034
:1036C0007000700070007F007F007F007F0070003E
:1036D00070007000E000E000E000FE00FE00FE0070
:1036E0003FC03FC03FC038007000700070007F8056
:1036F0007F807F807F80700070007000E000E000BD
:10370000E000E000E000E0000F003F803F8079C073
:1037100070C070C0F000E000E000E000E000E7C032
:10372000E7C0E7C0E1C0E1C0F3807F807F803E005A
:1037300038C038C038C038C038C0718071807180DE
:103740007F807F807F807F8071807180E300E300D5
:10375000E300E300E300E3000E000E000E000E00A5
:103760000E001C001C001C001C001C001C001C0087
:103770001C001C00380038003800380038003800C1
:1037800001C001C001C001C001C0038003800380EB
:10379000038003800380038003800380E700E70049
:1037A000E700FF00FF007E0039C039C03B803B804E
:1037B0003B00770077007E007C007C007C007E0070
:1037C000770073807380E380E1C0E1C0E1C0E1C0B5
:1037D0003800380038003800380070007000700081
:1037E0007000700070007000700070007000E000E9
:1037F000E000FF00FF00FF0031C031C031C031C028
:1038000031C079C07BC07BC07F807F807F807F801C
:103810007D807D806D80E980EB00EB00EB00E300B4
:1038200030C030C038C038C038C079807D807D80DD
:103830007D807F8077807780778077807780E700D2
:10384000E700E700E300E3000F003F803F807BC01C
:1038500071C071C0F1C0E1C0E1C0E1C0E1C0E1C030
:10386000E1C0E3C0E380E380F7807F007F003C009D
:103870003F803FC03FC039C039C071C071C073C004
:103880007F807F807F007F00700070007000E0000C
:10389000E000E000E00000000F003F803F807BC0C0
:1038A00071C071C0F1C0E1C0E1C0E1C0E1C0E1C0E0
:1038B000E3C0EB80EF80FF007F007B0033800000DF
:1038C0003F803FC03FC038C038C070C070C071C0BA
:1038D0007F807F807F007F007E007E007700E30096
:1038E000E300E380E18000001F003F803F8073C061
:1038F00071C071C0700078003E003E000F000F00E4
:103900000780E380E380E380F3807F007F003E0058
:10391000FFC0FFC0FFC00E000E001C001C001C00FA
:103920001C001C001C001C001C001C001C0038009B
:10393000380038003800380039C039C039C039C0C3
:1039400039C07380738073807380738073807380D9
:103950007380E700E700E700E700FE00FE007C0060
:10396000E0C0E0C0E1C0E1C0E1C07380738073805B
:1039700077007700770077007E007E007E003C00B5
:103980003C003C0038003000CCC0CCC0CCC0CCC027
:10399000DCC0DDC0DDC0DF80DF80FF807F8077801E
:1039A0007700770077007700760066006600660093
:1039B000E0C0E0C07180718073003E003E003C00BA
:1039C0001C001C003C003C003E006E006E00C70066
:1039D000870087808380038080C0C0C0C1C0C1C011
:1039E000C380E700E7006E007E007E003C003C00E4
:1039F00038003800380070007000700070007000EF
:103A00003FC03FC03FC0038003800700070007009E
:103A10000E000E001C001C0038003800380070003A
:103A20007000FF80FF80FF80000000001F001F006B
:103A30001F001C001C001C001C001C001C001C00A3
:103A40001C001C001C001C001C001F001F001F008D
:103A5000000000007000700070003800380038006E
:103A6000380038001C001C001C001C001C000E004C
:103A70000E000E0000000000000000001F001F00EC
:103A80001F000700070007000700070007000700E6
:103A9000070007000700070007001F001F001F00A6
:103AA00008001C003E003E0077007700E380E380C2
:103AB0000000000000000000000000000000000006
:103AC00000000000000000000000000000000000F6
:103AD00000000000000000000000000000000000E6
:103AE00000000000000000000000FFC0FFC0FFC099
:103AF00000001E000E000700030000000000000090
:103B000000000000000000000000000000000000B5
:103B100000000000000000000000000000000000A5
:103B2000000000001F003F803F8073C001C01F8065
:103B30007F807F80F380E780E700FF00FF00770051
:103B40003800380038003800380038003F807F8067
:103B50007F8079C071C071C071C071C0F1C0F38045
:103B6000F380FF00FF00EE000000000000000000F6
:103B7000000000000F003F803F8039C079C0700016
:103B8000F000F000E000E38077007F003F001E00BF
:103B900001C001C001C001C001C001C03DC07FC063
:103BA0007FC077806380E380E380E380C780C700C5
:103BB000EF007F007F0076000000000000000000A2
:103BC000000000000F001F803F8039C071C071C02D
:103BD000FFC0FFC0E000738073003F003F001E0085
:103BE0000780078007800E000E000E003F003F0098
:103BF0003F000E001C001C001C001C001C001C00D0
:103C000038003800380038000000000000000000D4
:103C100000001DC07FC073C073C0E3C0E380E780B5
:103C20007F007F0077000700CF00FE00FE007C00D1
:103C30003800380038003800380038003B807FC03A
:103C40007FC079C071C071C071C071C0E380E38072
:103C5000E380E380E380E3800700070007000700BC
:103C6000000000000E000E000E000E000E001C00F2
:103C70001C001C001C001C003800380038003800F4
:103C8000038003800380038000000000070007001A
:103C90000700070007000E000E000E000E000E00C9
:103CA0001C00FC00FC00F800380038003800380028
:103CB0003800380039C03380338077007E007E00C2
:103CC0007E007E0077007700E700E700E700E380F2
:103CD0000E000E000E000E000E000E000E001C0066
:103CE0001C001C001C001C001C001C0038003800BC
:103CF00038003800380038000000000000000000E4
:103D00000000000029807FC07FC076C064C064C00E
:103D100064C064C0E4C0C980C980C980C980C9804A
:103D20000000000000000000000000003B807FC099
:103D30007FC079C071C071C071C071C0E380E38081
:103D4000E380E380E380E3800000000000000000E7
:103D5000000000001F003F803F8073C0F1C0E1C041
:103D6000E1C0E1C0E1C0E380F3807F007F003E005E
:103D70000000000000000000000000003B803F80C9
:103D80003FC039C038C070C071C071C073807F80BF
:103D90006F00E000E000E000000000000000000014
:103DA000000000001DC03FC03FC073C061C0E1C043
:103DB000E380E380F7807F803B800380070007007B
:103DC0000000000000000000000000003B803FC039
:103DD0003FC03C4038007000700070007000700000
:103DE0007000E000E000E0000000000000000000C3
:103DF000000000000F001F801F8039C038003E0007
:103E00001F001F000780E380F3807F007F003E00DB
:103E100007000700070007000E000E003F003F00EC
:103E20003F001C001C001C001C001C003800380057
:103E300038003E003E001E000000000000000000B0
:103E400000000000F1C0F1C0F1C071C073C0738008
:103E5000E380E380E380E780E780FF00FF007700F6
:103E6000000000000000000000000000E1C0E3C00E
:103E7000E3C0E380E700E700EE00EE00EE007C0028
:103E80007C0078007800780000000000000000004E
:103E9000000000008CC0CCC0CCC0CCC0DD80DD8078
:103EA000D580D580F700F700E700E700E700E700DE
:103EB00000000000000000000000000071C07380DE
:103EC0003F003F003E001E001C003C003C003E0046
:103ED000FE00EF00C700C700000000000000000067
:103EE00000000000E1C0E1C0E380E3807380770060
:103EF0007E007C007C003C007800F000E000E000E8
:103F00000000000000000000000000003F803F8033
:103F10003F00070007000E001E001C001C003800B8
:103F200038007F007F007F0007000F001F001C008B
:103F30001C001C001C001C003C00780078003C00A9
:103F40001C001C001C001C001C001F000F000700B0
:103F50001C001C001C001C001C001C001C001C0081
:103F60001C001C001C001C001C001C001C001C0071
:103F70001C001C001C001C00700078007C001C0051
:103F80001C001C001C001C001E000F000F001E0067
:103F90001C001C001C001C001C007C007800700031
:103FA00000000000000078C0FDC0EFC0C780000026
:103FB0000000000000000000000000000000000001
:103FC00000000000000000000000000000000000F1
:103FD00000000000000000000000000000000000E1
:103FE00000000000000000000000000000000000D1
:103FF000FF00FF00FF007000700070007000700094
:104000007E007F007F8073807380738073807380F5
:1040100073807780770076000F003F003C0000003F
:10402000FF80FF80FF80E000E000E000E000E000B3
:10403000E000E000E000E000E000E000E000E00080
:104040000000000000000000000000000000000070
:104050000000000000000000000000003C003C00E8
:104060003C000C000C001800000000000F003F0096
:104070003C000000FF80FF80FF80E000E000E000E7
:10408000E000E000E000E000E000E000E000E00030
:104090000000000000000000000000000000000020
:1040A000000000000000000000000000F3C0F3C0AA
:1040B000F3C030C030C0618000000000000000008C
:1040C00000000000000000000000000000000000F0
:1040D00000000000000000000000EEE0EEE0EEE076
:1040E0000000000000001C001C001C001C00FF80E1
:1040F000FF80FF801C001C001C001C001C001C001A
:104100001C001C001C001C000000000000001C0023
:104110001C001C001C00FF80FF80FF801C001C0096
:104120001C00FF80FF80FF801C001C001C001C0086
:10413000000000001F003F807FC0F1C0E0C0E00031
:10414000FF00FF00E000E000FF00FF00E000E000F3
:10415000F1C07FC03F801F00000000000000000091
:104160007000704050C071C073C007800F001E0007
:104170003C00780070006EE04EE00AA00EE00EE019
:104180001F003F007F0077007700770077007700FF
:10419000778077C077E077E07760776077607760E7
:1041A00077E0F7E0E7C0C7800000000000000040B3
:1041B00000C001C0038007000E001C003800700022
:1041C00038001C000E000700038001C000C0004042
:1041D000EE00EE00EE00EE00EE00EE00EE00EE006F
:1041E000FF00FF80EFC0EFC0EEC0EEC0EEC0EEC03B
:1041F000EFC0EFC0EF80EF000F003F003C00000079
:10420000E180E380E700EE00FC00F800F000E00051
:10421000F000F800FC00EE00E700E380E1C0E0C041
:10422000FF80FF80FF8038003800380038003F00F2
:104230003F803FC039C039C039C039C039C039C0EA
:1042400039C039C039C039C0E1C0E1C0E1C0E1C006
:10425000E1C0E1C0E1C0E1C0FFC0FFC07F801E003F
:104260001E001E001E001E001E001E001E001E005E
:104270000000000038003800FF80FF80FF80380019
:10428000380038003F003F803BC039C039C039C0DA
:1042900039C03BC03F803F000C00180018001E00D2
:1042A0001E001E00000000000000000000000000D2
:1042B00000000000000000000000000000000000FE
:1042C0001E001E001E00060006000C00000000007C
:1042D00000000000000000000000000000000000DE
:1042E00000000000000000006180C300C300F3C0B4
:1042F000F3C0F3C000000000000000000000000058
:1043000000000000000000000000000000000000AD
:10431000F3C0F3C0F3C030C030C0618000000000C3
:10432000000000000000000000000000000000008D
:10433000000000000000000000000000000000007D
:1043400000000000000000001E003F003F003F0092
:104350003F001E0000000000000000000000000000
:10436000000000000000000000000000000000004D
:10437000000000003E003E003E0000000000000083
:10438000000000000000000000000000000000002D
:10439000000000000000000000000000FFC0FFC09F
:1043A000FFC000000000000000000000000000004E
:1043B00000000000000000000000000000000000FD
:1043C00000000000000000000000000000000000ED
:1043D00000000000000000000000FC4026C027C0D4
:1043E00025402440244000000000000000000000A0
:1043F00000000000000000000000000000000000BD
:10440000000000000000000000001F003F007F00CF
:1044100077007700778077C077E0776077607760A4
:104420007760F7E0E7C0C780000000000000800070
:10443000C000E000700038001C000E000700038080
:1044400007000E001C0038007000E000C000800073
:1044500000000000000000000000EE00EE00EE0092
:10446000EE00EE00FF00FF80FFC0EFC0EEC0EEC028
:10447000EFC0EFC0EF80EF00000000001E007E00E4
:1044800078000000E380E700EE00FC00F800F00098
:10449000E000F000F800FC00EE00E700E380E1C07F
:1044A0000000000070007000F800F800F8007000D4
:1044B000700077007F807FC07BC071C071C071C009
:1044C00071C071C071C071C0000000000000000028
:1044D0000000E1C0E1C0E1C0E1C0E1C0E1C0E1C075
:1044E000E1C0FFC0FFC07F801E001E001E001E0036
:1044F00000000000000000000000000000000000BC
:1045000000000000000000000000000000000000AB
:10451000000000000000000061807F801E00E1C0FC
:10452000E1C0E1C0E1C0E1C0E1C0F3C073807F80C1
:104530003F003F001E001E003E00FC00F800F0009F
:1045400000000000000061807F801E00E1C0E1C02B
:10455000E1C0E1C073807F803F003F001E001E006D
:104560003E00FC00F800F00003800380038003801D
:104570000380038003800380038003800380038023
:10458000038003800380E380F780FF807F003E008C
:10459000000000000000000000000000C0C0EDC0EE
:1045A0007F8033006180618033007F80EDC0C0C0B8
:1045B000000000000000000001C001C0FFC0FFC0FB
:1045C000FFC0E000E000E000E000E000E000E0000C
:1045D000E000E000E000E000E000E000E000E000DB
:1045E000000000003800380038003800380038007B
:1045F000380038000000000038003800380038006B
:1046000038003800380038003E007F00FF80E3802B
:10461000E180F0007E007F00FF80E380E380FF8088
:104620007F003F000780C380E380FF807F003E0063
:10463000330033000000FF80FF80FF80E080E00057
:10464000E000FE00FE00FE00E000E000E000E00010
:10465000E000FF80FF80FF800000000000000000FD
:104660003F807FC0FFE0E0E0CE60DF60DB60D860CD
:10467000DB60DF60CE60E0E0FFE07FC03F800000F5
:104680001F003F807FC0F1C0E000E000E000FF00BD
:10469000FF00FF00E000E000E000E000E000E000DC
:1046A000F1C07FC03F801F0000000000000000003C
:1046B000000000000000084018C039C07380E70007
:1046C000738039C018C008400000000000000000DE
:1046D00000000000000000000000000000000000DA
:1046E000000000000000000000000000FFC0FFC04C
:1046F000FFC001C001C00000000000000000000079
:1047000000000000000000007F807F807F800000AC
:104710000000000000000000000000000000000099
:10472000000000003F807FC0FFE0E0E0C060DE608E
:10473000DF60DB60DB60DF60DE60DF60DB60C060AD
:10474000E0E0FFE07FC03F801B001B0000000E0088
:104750000E000E000E000E000E000E000E000E00E9
:104760000E000E000E000E000E000E000E000E00D9
:1047700000001B003B003B8071C071C03B801B00F0
:104780001B0000000000000000000000000000000E
:104790000000000000000000000000000000000019
:1047A0000E000E000E007FC07FC07FC00E000E0006
:1047B0000E0000007FC07FC07FC00000000000002E
:1047C0000E000E000E000E000E000E000E000E0079
:1047D0000E000E000E000E000E000E000E000E0069
:1047E0000E000E000E000E0000001C001C001C003D
:1047F00000001C001C001C001C001C001C001C00F5
:104800001C001C001C001C001C001C001C001C00C8
:1048100000000000000001C001C0FFC0FFC0FFC0D9
:10482000E000E000E000E000E000E000E000E00088
:10483000E000E000E000E0000000000000000000F8
:104840000000E380E380E380E380E380E380E380B3
:10485000F780FF80FF80EB80E000E000E000E000F8
:10486000000000003FC07FC0FFC0FDC0FDC0FDC014
:10487000FDC0FDC07DC03DC01DC01DC01DC01DC010
:104880001DC01DC01DC01DC00000000000000000B4
:1048900000000000000000001E001E001E001E00A0
:1048A0000000000000000000000000000000000008
:1048B000000033003300000000003F007F80FFC095
:1048C000F3C0E1C0E1C0FFC0FFC0FF80E000E00036
:1048D000F1C0FFC07F803F00C600C600C600C60012
:1048E000C600E600E600F680FFC0DFC0CF40CF4044
:1048F000C740C7C0C7C0C680C600C7C0C7C0C7C002
:10490000000000000000000000003F007F80FFC0AA
:10491000F1C0E000E000FE00FE00FE00E000E0006C
:10492000F1C0FFC07F803F000000000000000000D9
:10493000000000000000000000008400C600E70046
:10494000738039C07380E700C60084000000000057
:1049500001C001C001C0000001C001C001C001C010
:1049600001C001C001C001C001C001C001C071C0CF
:104970007BC07FC03F801F001E003F007F80F38010
:10498000E000E000E000F0007E003F001F8003C078
:1049900001C000C001C0C1C0E3C0FF807F003E0075
:1049A000000000000000000000003F007F80FFC00A
:1049B000F1C0E000F000FF007F803FC003C0C1C035
:1049C000E3C0FFC07F803F00000000001B001B0011
:1049D000000000000E000E000E000E000E000E0083
:1049E0000E000E000E000E000E000E000E000E0057
:1049F0000780078007800F800F800F801D801D803B
:104A00001D801D801D80398039807F807FC07FC0E0
:104A1000E1C0E1C0E1C0C1C03FC03FC03FC03800FD
:104A200070007000700070007F807F807FC071C058
:104A300070C070C0E0C0E1C0E1C0FF80FF00FF00B7
:104A40003F803FC03FC039C071C071C073C07F801C
:104A50007F007F807F80738071C071C0E1C0E1C042
:104A6000E3C0FF80FF80FF003FC03FC03FC0380071
:104A700070007000700070007000700070007000B6
:104A800070007000E000E000E000E000E000E00006
:104A90000FC00FC00EC00EC00EC00D801D801D8047
:104AA0001D801D80398039803B003B003B00730036
:104AB000FF80FF80C380C3803FC03FC03FC038003D
:104AC00038007000700070007F807F807F807F8062
:104AD00070007000E000E000E000FF00FF00FF0059
:104AE00066406640664076C0378037803F803F0032
:104AF0003F001E003E003E007F007F007F00DB0085
:104B0000DB80DB80D980D9800F800F801FC03DC043
:104B100039C001C001C003C00F800F000F00038027
:104B2000038003806380E380F7807F007F003E0086
:104B300038C038C039C039C03BC0738077807F80AF
:104B40007D807D807980718071807180E300E300D9
:104B5000E300E300E300E3000CC00FC0030038C033
:104B600038C039C039C03BC0738077807F807D807A
:104B70007D807980718071807180E300E300E300C3
:104B800039C039C03B803B803B00770077007E0016
:104B90007C007C007C007E007700738073807380D3
:104BA000E380E1C0E1C0E1C01FC01FC01FC01CC046
:104BB0001CC039803980398039803980398039800A
:104BC00039803980398073007300F300E300E3001B
:104BD00031C031C031C031C031C079C07BC07BC071
:104BE0007F807F807F807F807D807D806D80E98079
:104BF000E980EB00EB00E30038C038C038C038C0B3
:104C000038C07180718071807F807F807F807F80DD
:104C100071807180E300E300E300E300E300E30060
:104C20000F003F803F807BC071C071C0F1C0E1C008
:104C3000E1C0E1C0E1C0E1C0E3C0E380E380E38024
:104C4000F7807F007F003C003FC03FC03FC038C0BE
:104C500038C038C0718071807180718071807180BE
:104C600071807180E300E300E300E300E300E30010
:104C70003F803FC03FC039C039C071C071C073C0F0
:104C80007F807F807F007F0070007000E000E00088
:104C9000E000E000E000E0000F003F803F807BC0CC
:104CA00071C071C0F000E000E000E000E000E00052
:104CB000E000E000E380E380F7007F007F003C003D
:104CC000FFC0FFC0FFC00E000E001C001C001C0037
:104CD0001C001C001C001C001C001C0038003800BC
:104CE0003800380038003800604060C061C061C0E2
:104CF000338033803380370036003E003E003C0076
:104D00003C003C00380070007000F000E000E00063
:104D100006000600060006001F001F007F806DC011
:104D20006DC0CCC0CCC0CCC0CCC0ED807F807F80BB
:104D30003E00180018001800E0C0E0C071807180CB
:104D400073003E003E003C001C001C003C003C0088
:104D50003E006E006E006700C700C780C38083807E
:104D600038C038C038C038C038C038C07180718091
:104D700071807180718071807180E300E300FF8039
:104D8000FF80FF800180018071C071C071C071C05F
:104D900071C0E380E380E380E380E380FF807F8075
:104DA0007B8003800700070007000700070007005B
:104DB00036C036C036C036C036C06D806D806D805E
:104DC0006D806D806D806D806D806D80DB00DB009F
:104DD000DB00FF00FF00FF0036C036C036C036C023
:104DE00036C06D806D806D806D806D806D806D8052
:104DF000DB00DB00DB00FF00FF00FF00038003801F
:104E0000F800F800F8003800380038007000700032
:104E10007F807F807FC071C071C071C071C0E1C0F0
:104E2000E380FF80FF00FF0038C038C038C038C0C2
:104E300038C038C0718071807D807D807E807680B2
:104E4000768076807580E500ED00FB00FB00FB00BE
:104E50003800380038003800380038007000700022
:104E60007F807F807FC071C071C071C071C0E1C0A0
:104E7000E380FF80FF00FF001F001F003F803BC05A
:104E80003BC071C001C001C00FC00FC00FC001C046
:104E900001C001C001C06380F780FF807F003C003B
:104EA00033003380378037C037C037C06DC06DC026
:104EB0006DC079C079C079C07BC07BC07BC06F807A
:104EC000CF80CF00CF00C6000FC01FC01FC018C0CA
:104ED00038C03980398039801F801F8007800F805B
:104EE0000F801D803B003B0033007700E700E700A8
:104EF0000000000000000000000000001F003F80D4
:104F00003F8073C001C01F807F807F80F380E78077
:104F1000E700FF00FF00770000C007C00F801F8080
:104F20001800180036003E003F007F807B807380B1
:104F30007380E700E700E700EF00FE00FE007C0062
:104F40000000000000000000000000003F803FC0A3
:104F50003FC039C073C07F807F807F8071C071C0C7
:104F6000E3C0FF80FF80FF000000000000000000A1
:104F7000000000003FC03FC03FC03800700070001C
:104F80007000700070007000E000E000E000E000E1
:104F90000000000000000000000000000FC00FC073
:104FA0000EC01EC01D801D80398039803B007300FB
:104FB000FF80FF80C380C38000000000000000006D
:104FC000000000000F001F803F8039C071C071C019
:104FD000FFC0FFC0E000E380F3007F003F001E0041
:104FE0000000000000000000000000006640664075
:104FF00076C0378037803F803F001E003E003E0075
:105000007F00DB00DB80D980000000000000000092
:10501000000000000F800F801FC03DC039C003C0DA
:105020000F800F000F006380F7807F007F003E003D
:1050300000000000000000000000000038C039C07F
:1050400039C03BC0738077807F807D807D80798090
:10505000E300E300E300E3000000000000000CC0F8
:105060000FC0030038C039C039C03BC0738077809F
:105070007F807D807D807980E300E300E300E300B2
:1050800000000000000000000000000039C0338074
:10509000338077007E007E007E007E007700770000
:1050A000E700E700E700E3800000000000000000E8
:1050B000000000001FC01FC01FC01CC03980398005
:1050C00039803980398073007300F300E300E30016
:1050D00000000000000000000000000031C031C0EE
:1050E00031C079C07BC07BC07F807F807D807D8028
:1050F0006D80E980EB00E30000000000000000008C
:105100000000000038C038C038C038C071807F80CF
:105110007F807F807F807180E300E300E300E30015
:105120000000000000000000000000001F003F80A1
:105130003F8073C0F1C0E1C0E1C0E1C0E1C0E380E5
:10514000F3807F007F003E000000000000000000B0
:10515000000000003FC03FC03FC038C07180718078
:105160007180718071807180E300E300E300E300EF
:105170000000000000000000000000003B803F80B5
:105180003FC039C038C070C071C071C073807F80AB
:105190006F00E000E000E000000000000000000000
:1051A000000000000F003F803F8039C079C07000D0
:1051B000E000E000E000E380F700FF007F003E0039
:1051C000000000000000000000000000FFC0FFC061
:1051D000FFC00E001C001C001C001C001C001C005A
:1051E0001C003800380038000000000000000000FB
:1051F00000000000E1C0E1C0E380E380738077003D
:105200007E007C007C003C007800F000E000E000C4
:105210000000000000000000000000000600060082
:105220001F001F007F806DC0CCC0CCC0ED807F8090
:105230007F803E0018001800000000000000000001
:105240000000000071C073803F003F003E001E0060
:105250001C003C003C003E00FE00EF00C700C70001
:1052600000000000000000000000000038C038C04E
:1052700038C038C07180718071807180E300FF8018
:10528000FF80FF800180018000000000000000001E
:105290000000000071C071C071C071C0E380E38084
:1052A000E380FF807F807B8003800700070007008A
:1052B00000000000000000000000000036C036C002
:1052C00036C036C06D806D806D806D806D80DB0076
:1052D000DB00FF00FF00FF000000000000000000F6
:1052E0000000000036C036C036C06D806D806D8015
:1052F0006D806D80DB00FF00FF00FF00038001C0B8
:10530000000000000000000000000000F800F800AD
:10531000F800380070007F807FC071C0E1C0E3807A
:10532000FF80FF00FF000000000000000000000000
:105330000000000038C038C038C0718071807D80A6
:105340007D807680E500ED00FB00FB00FB000000A7
:1053500000000000000000000000000038003800DD
:105360003800380070007F807FC071C0E1C0E380EA
:10537000FF80FF00FF0000000000000000000000B0
:10538000000000001F001F003F803BC071C001C033
:105390000FC00FC06380F780FF807F003C000000DB
:1053A0000000000000000000000000003300338017
:1053B000378037C037C06DC079C07BC07BC06F807D
:1053C000CF80CF00C60000000000000000000000F9
:1053D000000000000FC01FC01FC038C039801F80F0
:1053E0001F8007800F801D803B007300E7000000D6
:1053F00000000000000000000000000000000000AD
:10540000000000000000000000000000000000009C
:10541000000000000000000000000000000000008C
:10542000000000000000000000000000000000007C
:10543000000000000000000000000000000000006C
:10544000000000000000000000000000000000005C
:10545000000000000000000000000000000000004C
:10546000000000000000000000000000000000003C
:10547000000000000000000000000000000000002C
:10548000000000000000000000000000000000001C
:10549000000000000000000000000000000000000C
:1054A00000000000000000000000000000000000FC
:1054B00000000000000000000000000000000000EC
:1054C00000000000000000000000000000000000DC
:1054D00000000000000000000000000000000000CC
:1054E00000000000000000000000000000000000BC
:1054F00000000000000000000000000000000000AC
:10550000000000000000000000000000000000009B
:10551000000000000000000000000000000000008B
:10552000000000000000000000000000000000007B
:10553000000000000000000000000000000000006B
:10554000000000000000000000000000000000005B
:10555000000000000000000000000000000000004B
:10556000000000000000000000000000000000003B
:10557000000000000000000000000000000000002B
:10558000000000000000000000000000000000001B
:10559000000000000000000000000000000000000B
:1055A0000000000000000000C060C060E0E0E0E03B
:1055B00071C071C03B803B801F001F000E001F00A8
:1055C0001F003B803B8071C071C0E0E0E0E0C06044
:1055D00000000000000000000000000000000000CB
:1055E00000000000000000000000000000000000BB
:1055F00000000000000000000000000000000000AB
:10560000000000000000000000000000000000009A
:1058C0000000000000000000000000000000FFC019
:1058D000FFC0FFC0000000000000FFC0FFC0FFC00D
:1058E000000000000000FFC0FFC0FFC0000000007B
:1058F00000000000000000000000000000000000A8
:105900000000000000000000000000000000000097
:10591000000000000000000000000C001E001E003F
:105920001E001E001E001E001E001E001E001E0087
:105930000C00000000001E001E001E001E000000E3
:10594000F3C0F3C0F3C0F3C0F3C071C06180C30003
:1059500082000000000000000000000000000000C5
:1059600000000000000000001980198019801980D3
:105970003300FFC0FFC0FFC0330033006600FFC02C
:10598000FFC0FFC0660066006600CC00CC000000CF
:105990000C003F007F80FFC0EDC0EDC0EC00EC00CC
:1059A0007C007F003F800FC00DC0EDC0EDC0EDC09A
:1059B0007F807F803F000C007000F8C0D9C0F9C024
:1059C00073800380070007000E000E001C001C00FF
:1059D0003800380070007380E7C0E6C0C7C003809D
:1059E0001E003F007F807380738073807F803F0044
:1059F0001E003E007C00FEC0F7C0E3C0E380E380F1
:105A0000F780FFC07FC03CC01E001E001E001E00AD
:105A10001E000E000E001C00180000000000000018
:105A20000000000000000000000000000000000076
:105A300003000F000E001C001C003C003800380062
:105A40003800380038003800380038003C001C00AE
:105A50001C000E000F00030030003C001C000E0074
:105A60000E000F00070007000700070007000700EF
:105A7000070007000F000E000E001C003C00300065
:105A80000000000000000C001E001E00CCC0FFC083
:105A9000FFC0DE401F007F807380330000000000E5
:105AA0000000000000000000000000001E001E00BA
:105AB0001E001E00FFC0FFC0FFC0FFC01E001E0072
:105AC0001E001E000000000000000000000000009A
:105AD00000000000000000000000000000000000C6
:105AE0000000000000001E001E001E001E001E0020
:105AF0000E000E001C001800000000000000000056
:105B000000000000FFC0FFC0FFC0FFC00000000099
:105B10000000000000000000000000000000000085
:105B20000000000000000000000000000000000075
:105B30000000000000000000000000001E003F0008
:105B40003F003F003F001E00000000C001C001C038
:105B500003800380070007000E000E001C001C00DD
:105B60003800380070007000E000E000C000000065
:105B70001E0033002100618061806180E1C0E1C0CE
:105B8000E1C0E1C0E1C0E1C0E1C0E1C0618061808D
:105B90006180210033001E0004000C003C007C00EA
:105BA0001C001C001C001C001C001C001C001C0015
:105BB0001C001C001C001C001C001C001C007F00A2
:105BC0001E007F007F004780838083800380030066
:105BD0000300030006000C000C00080010401040F9
:105BE0003FC07F807F80FF801F803FC03FC063C079
:105BF00001C001C001800300030007C003E001E011
:105C000001E000E000E000E060C0718073803F00D0
:105C10000180018001800380078007800B800B805A
:105C20000B801380238043808380FFC0FFC0FFC0B0
:105C300003800380038003801FC03FC03FC03F80BC
:105C40004000400078007F007F00FF8003C000C05C
:105C500000C0004000400040E040F080F1807F0044
:105C600001C007000F003C00300070007000FF0012
:105C7000FF00E380E1C0E1C0E1C0E1C0E1C0E1C0FC
:105C800061C0718073801F007FC07FC07FC07F8034
:105C9000C180C1808180030003000300030006006F
:105CA000060006000C000C000C000C001C00180084
:105CB0003E0073007300E180E180E180F100730039
:105CC0007F003F003F8063C063C0C1C0C1C0C1C08E
:105CD000C1C0638063803F001E00338033807180C9
:105CE00071C071C071C071C071C071C039C01F80F6
:105CF0001F8003800300030007001C001C007000CD
:105D00000000000000003C003C003C003C000000A3
:105D100000000000000000003C003C003C003C0093
:105D200000000000000000000000000000003C0037
:105D30003C003C003C0000000000000000000000AF
:105D40003C003C003C003C000C001C003800000003
:105D5000000000800180038007800F001E003C00CF
:105D60007800F000E000F00078003C001E000F001A
:105D70000780038001800080000000000000000018
:105D80000000FF80FF80FF80000000000000FF8017
:105D9000FF80FF8000000000000000000000000005
:105DA000000040006000700078003C001E000F0002
:105DB000078003C001C003C007800F001E003C0025
:105DC00078007000600040001E003F007F80F3807C
:105DD000E3C0E1C0E1C001C001C003C0038007808F
:105DE0000F001E001C00000000001C001C001C0016
:105DF0003F007F80FFC0E1C0CCC0DEC0DEC0D2C0AB
:105E0000D2C0D2C0D2C0D2C0DEC0DEC0CF80C700F8
:105E1000E040FFC07FC03F800400040006000E0089
:105E20000E000F000F0017001700170017001700D3
:105E300023803F803F802380238023C0F7E0F7E06A
:105E4000FF00FF8039C038E038E038E038E039C082
:105E50003F803F8039C039C038E038E038E038E072
:105E600038E039C0FF80FF000F201F2038E070604D
:105E7000706060206020E000E000E000E000E000F2
:105E8000E000E000E0007020702038401F800F002C
:105E9000FC00FE003B8039C039C038C038C038E053
:105EA00038E038E038E038E038E038E038E039C051
:105EB00039C03B80FE00FC00FFC0FFC038C0384046
:105EC00038403A003A003A003E003E003A003A00BC
:105ED0003A0038203820382038203860FFE0FFE0D2
:105EE000FFE0FFE038603820382039003900390001
:105EF0003F003F00390039003900380038003800D1
:105F000038003800FE00FE000E400E4039C070C060
:105F100070C070407040E000E000E000E000E00091
:105F2000E7E0E1C0E1C071C071C039C00F000E00F0
:105F3000FBE0FBE071C071C071C071C071C071C085
:105F40007FC07FC071C071C071C071C071C071C0AD
:105F500071C071C0FBE0FBE03F803F800E000E008F
:105F60000E000E000E000E000E000E000E000E00C1
:105F70000E000E000E000E000E000E003F803F804F
:105F80001FC01FC007000700070007000700070029
:105F900007000700070007000700E700E700E70029
:105FA000E700C6003C003C00F9C0F9C070807300F7
:105FB00073007200720074007C007C007E007E0022
:105FC0007700770077007380738071C0F9E0F9E0A3
:105FD000FE00FE0038003800380038003800380075
:105FE0003800380038003800380038203820382091
:105FF00038203860FFE0FFE0E3E0E3E063C073C017
:1060000073C073C073C073C075C075C075C075C0F0
:1060100079C079C059C059C049C049C0EBE0EBE034
:10602000E3E0E3E070807880788078807C805C803A
:106030005E804E804E804E80478047804780438000
:1060400043804180F080F0800E001F003B8071C0D3
:1060500071C060C060C0E0E0E0E0E0E0E0E0E0E00F
:10606000E0E060C060C071C071C03B801F000E00E6
:10607000FF80FF8039C038E038E038E038E038E0B1
:1060800039C039C03F803F803800380038003800C0
:1060900038003800FE00FE000E001F003B8071C07B
:1060A00071C060C060C0E0E0E0E0E0E0E0E0E0E0BF
:1060B000E0E060C063C073C071803BE01FE00E6031
:1060C000FF80FF8039C038E038E038E038E038E061
:1060D00039C039C03F003F003F003F003F003B80D8
:1060E0003B8039C0FEE0FEE01E403F4060C0E04023
:1060F000E040E040E040F0007F007F001FC01FC094
:1061000081E080E080E0C0E0C0E0E0C09F808F00E0
:10611000FFE0FFE08E208E208E200E000E000E008D
:106120000E000E000E000E000E000E000E000E00FF
:106130000E000E003F803F80FDE0FDE0388038809B
:10614000388038803880388038803880388038808F
:10615000388038803880388038801D000E000E006E
:10616000FDE0FDE0704038803880388038803900AC
:1061700039003900190019001B001B001F001E0008
:106180000E000E0004000400F8E0F8E070407040DB
:106190007240734073407740774077407540754058
:1061A000754039C039C039C039C039C0108010803D
:1061B000F9E0F9E03080190019001A001A001E00F9
:1061C0000E000E000E000E000F000B000B0013005F
:1061D00013002180F3E0F3E0FDE0FDE07040384083
:1061E0003840388038801C801D001D001E001E00B5
:1061F0000E000E000E000E000E000E003F803F80CD
:106200007FC07FC0638047004700470047000E0003
:106210001C001C001C001C003800382038203820CE
:1062200038207060FFE0FFE0000000001F001F004A
:106230001F001C001C001C001C001C001C001C007B
:106240001C001C001C001C001C001F001F001F0065
:106250000000000070007000700038003800380046
:10626000380038001C001C001C001C001C000E0024
:106270000E000E0000000000000000001F001F00C4
:106280001F000700070007000700070007000700BE
:10629000070007000700070007001F001F001F007E
:1062A00008001C003E003E0077007700E380E3809A
:1062B00000000000000000000000000000000000DE
:1062C00000000000000000000000000000000000CE
:1062D00000000000000000000000000000000000BE
:1062E00000000000000000000000FFC0FFC0FFC071
:1062F00000001E000E000700030000000000000068
:10630000000000000000000000000000000000008D
:10631000000000000000000000000000000000007D
:10632000000000003F006380C380C380C3800380FF
:106330001F807F80E380E380E380E780E78079C08F
:10634000F0007000700070007000700077007B80BB
:106350007B8071C071C071C071C071C071C071C0EB
:1063600071807B807B804F000000000000000000F7
:10637000000000001F8073C071C061C0E000E00039
:10638000E000E000E000E000E00070C079801F0065
:106390000780038003800380038003803B80778035
:1063A0007780E380E380E380E380E380E380E38041
:1063B000E38077C077C03B000000000000000000D1
:1063C000000000007E00C300C300C380C380FF80C4
:1063D000FF80C000C000C000C080E180F3003E002C
:1063E0000F003B803B803B00380038007C003800C9
:1063F00038003800380038003800380038003800DD
:106400003800380038007C00000000000000000068
:10641000000000007F80C600C700C700C700C6009C
:106420007C008000FF00FF80FF8000800100FE00F4
:10643000F00070007000700070007000778079C00C
:1064400079C071C071C071C071C071C071C071C0BC
:1064500071C071C071C0F9E00E000E000E000E0098
:10646000000000001E000E000E000E000E000E00C8
:106470000E000E000E000E000E000E000E001F009B
:1064800003800380038003800000000007800380F6
:1064900003800380038003800380038003800380E4
:1064A000638063803F001E00F00070007000700089
:1064B0007000700073C07180718071007200740090
:1064C00074007E0077007700738071C071C0FBE0BC
:1064D0001E000E000E000E000E000E000E000E003C
:1064E0000E000E000E000E000E000E000E000E003C
:1064F0000E000E000E001F00000000000000000053
:1065000000000000E98076C076C064C064C064C04A
:1065100064C064C064C064C064C064C064C0E4E0BB
:10652000000000000000000000000000F78079C0BB
:1065300079C071C071C071C071C071C071C071C0CB
:1065400071C071C071C0F9E00000000000000000DF
:10655000000000003F00738073806180E1C0E1C0F3
:10656000E1C0E1C0E1C0E1C06180738073803F00A1
:10657000000000000000000000000000F7007B8029
:1065800071C071C071C071C071C071C07B80770073
:10659000700070007000F8000000000000000000B3
:1065A000000000001C8073806380E380E380E38050
:1065B000E380E38077803B8003800380038007C013
:1065C000000000000000000000000000F7C07CC0D8
:1065D00078C0704070007000700070007000700033
:1065E000700070007000F800000000000000000063
:1065F000000000003EC061C0E1C0E0C0F800FE0045
:106600007F003F8007C003C0C1C0E1C0E180DF0060
:106610000400040004000C001C001C003F001C00CF
:106620001C001C001C001C001C001C001C001C008A
:106630001C001C801C800F000000000000000000F7
:1066400000000000F3C071C071C071C071C071C0A2
:1066500071C071C071C071C071C073C073C03DE0C2
:10666000000000000000000000000000F9E070C021
:1066700070C0388038803980398039801B001B0019
:106680001F000E000E0004000000000000000000CB
:1066900000000000FAE0724072407340774077409B
:1066A000774077403B803B803B80398039801100C8
:1066B000000000000000000000000000FBC07100AE
:1066C00071003A003C001C001C000E000E000F0080
:1066D000170023802380F7C00000000000000000A6
:1066E00000000000F9C07080388039001D001E00D5
:1066F0001E000E000C0004000800E800E800700016
:10670000000000000000000000000000FF000E007C
:106710000E000E001C001C0038007000700070009D
:10672000E100C100C100FF0007000F001F001C00B6
:106730001C001C001C001C003C00780078003C0081
:106740001C001C001C001C001C001F000F00070088
:106750001C001C001C001C001C001C001C001C0059
:106760001C001C001C001C001C001C001C001C0049
:106770001C001C001C001C00700078007C001C0029
:106780001C001C001C001C001E000F000F001E003F
:106790001C001C001C001C001C007C007800700009
:1067A00000000000000078C0FDC0EFC0C7800000FE
:1067B00000000000000000000000000000000000D9
:1067C00000000000000000000000000000000000C9
:1067D00000000000000000000000000000000000B9
:1067E00000000000000000000000000000000000A9
:1067F000FF00FF00FF00700070007000700070006C
:106800007E007F007F8073807380738073807380CD
:1068100073807780770076000F003F003C00000017
:10682000FF80FF80FF80E000E000E000E000E0008B
:10683000E000E000E000E000E000E000E000E00058
:106840000000000000000000000000000000000048
:106850000000000000000000000000003C003C00C0
:106860003C000C000C001800000000000F003F006E
:106870003C000000FF80FF80FF80E000E000E000BF
:10688000E000E000E000E000E000E000E000E00008
:1068900000000000000000000000000000000000F8
:1068A000000000000000000000000000F3C0F3C082
:1068B000F3C030C030C06180000000000000000064
:1068C00000000000000000000000000000000000C8
:1068D00000000000000000000000EEE0EEE0EEE04E
:1068E0000000000000001C001C001C001C00FF80B9
:1068F000FF80FF801C001C001C001C001C001C00F2
:106900001C001C001C001C000000000000001C00FB
:106910001C001C001C00FF80FF80FF801C001C006E
:106920001C00FF80FF80FF801C001C001C001C005E
:10693000000000001F003F807FC0F1C0E0C0E00009
:10694000FF00FF00E000E000FF00FF00E000E000CB
:10695000F1C07FC03F801F00000000000000000069
:106960007000704050C071C073C007800F001E00DF
:106970003C00780070006EE04EE00AA00EE00EE0F1
:106980001F003F007F0077007700770077007700D7
:10699000778077C077E077E07760776077607760BF
:1069A00077E0F7E0E7C0C78000000000000000408B
:1069B00000C001C0038007000E001C0038007000FA
:1069C00038001C000E000700038001C000C000401A
:1069D000EE00EE00EE00EE00EE00EE00EE00EE0047
:1069E000FF00FF80EFC0EFC0EEC0EEC0EEC0EEC013
:1069F000EFC0EFC0EF80EF000F003F003C00000051
:106A0000E180E380E700EE00FC00F800F000E00029
:106A1000F000F800FC00EE00E700E380E1C0E0C019
:106A2000FF80FF80FF8038003800380038003F00CA
:106A30003F803FC039C039C039C039C039C039C0C2
:106A400039C039C039C039C0E1C0E1C0E1C0E1C0DE
:106A5000E1C0E1C0E1C0E1C0FFC0FFC07F801E0017
:106A60001E001E001E001E001E001E001E001E0036
:106A70000000000038003800FF80FF80FF803800F1
:106A8000380038003F003F803BC039C039C039C0B2
:106A900039C03BC03F803F000C00180018001E00AA
:106AA0001E001E00000000000000000000000000AA
:106AB00000000000000000000000000000000000D6
:106AC0001E001E001E00060006000C000000000054
:106AD00000000000000000000000000000000000B6
:106AE00000000000000000006180C300C300F3C08C
:106AF000F3C0F3C000000000000000000000000030
:106B00000000000000000000000000000000000085
:106B1000F3C0F3C0F3C030C030C06180000000009B
:106B20000000000000000000000000000000000065
:106B30000000000000000000000000000000000055
:106B400000000000000000001E003F003F003F006A
:106B50003F001E00000000000000000000000000D8
:106B60000000000000000000000000000000000025
:106B7000000000003E003E003E000000000000005B
:106B80000000000000000000000000000000000005
:106B9000000000000000000000000000FFC0FFC077
:106BA000FFC0000000000000000000000000000026
:106BB00000000000000000000000000000000000D5
:106BC00000000000000000000000000000000000C5
:106BD00000000000000000000000FC4026C027C0AC
:106BE0002540244024400000000000000000000078
:106BF0000000000000000000000000000000000095
:106C0000000000000000000000001F003F007F00A7
:106C100077007700778077C077E07760776077607C
:106C20007760F7E0E7C0C780000000000000800048
:106C3000C000E000700038001C000E000700038058
:106C400007000E001C0038007000E000C00080004B
:106C500000000000000000000000EE00EE00EE006A
:106C6000EE00EE00FF00FF80FFC0EFC0EEC0EEC000
:106C7000EFC0EFC0EF80EF00000000001E007E00BC
:106C800078000000E380E700EE00FC00F800F00070
:106C9000E000F000F800FC00EE00E700E380E1C057
:106CA0000000000070007000F800F800F8007000AC
:106CB000700077007F807FC07BC071C071C071C0E1
:106CC00071C071C071C071C0000000000000000000
:106CD0000000E1C0E1C0E1C0E1C0E1C0E1C0E1C04D
:106CE000E1C0FFC0FFC07F801E001E001E001E000E
:106CF0000000000000000000000000000000000094
:106D00000000000000000000000000000000000083
:106D1000000000000000000061807F801E00E1C0D4
:106D2000E1C0E1C0E1C0E1C0E1C0F3C073807F8099
:106D30003F003F001E001E003E00FC00F800F00077
:106D400000000000000061807F801E00E1C0E1C003
:106D5000E1C0E1C073807F803F003F001E001E0045
:106D60003E00FC00F800F0000380038003800380F5
:106D700003800380038003800380038003800380FB
:106D8000038003800380E380F780FF807F003E0064
:106D9000000000000000000000000000C0C0EDC0C6
:106DA0007F8033006180618033007F80EDC0C0C090
:106DB000000000000000000001C001C0FFC0FFC0D3
:106DC000FFC0E000E000E000E000E000E000E000E4
:106DD000E000E000E000E000E000E000E000E000B3
:106DE0000000000038003800380038003800380053
:106DF0003800380000000000380038003800380043
:106E000038003800380038003E007F00FF80E38003
:106E1000E180F0007E007F00FF80E380E380FF8060
:106E20007F003F000780C380E380FF807F003E003B
:106E3000330033000000FF80FF80FF80E080E0002F
:106E4000E000FE00FE00FE00E000E000E000E000E8
:106E5000E000FF80FF80FF800000000000000000D5
:106E60003F807FC0FFE0E0E0CE60DF60DB60D860A5
:106E7000DB60DF60CE60E0E0FFE07FC03F800000CD
:106E80001F003F807FC0F1C0E000E000E000FF0095
:106E9000FF00FF00E000E000E000E000E000E000B4
:106EA000F1C07FC03F801F00000000000000000014
:106EB000000000000000084018C039C07380E700DF
:106EC000738039C018C008400000000000000000B6
:106ED00000000000000000000000000000000000B2
:106EE000000000000000000000000000FFC0FFC024
:106EF000FFC001C001C00000000000000000000051
:106F000000000000000000007F807F807F80000084
:106F10000000000000000000000000000000000071
:106F2000000000003F807FC0FFE0E0E0C060DE6066
:106F3000DF60DB60DB60DF60DE60DF60DB60C06085
:106F4000E0E0FFE07FC03F801B001B0000000E0060
:106F50000E000E000E000E000E000E000E000E00C1
:106F60000E000E000E000E000E000E000E000E00B1
:106F700000001B003B003B8071C071C03B801B00C8
:106F80001B000000000000000000000000000000E6
:106F900000000000000000000000000000000000F1
:106FA0000E000E000E007FC07FC07FC00E000E00DE
:106FB0000E0000007FC07FC07FC000000000000006
:106FC0000E000E000E000E000E000E000E000E0051
:106FD0000E000E000E000E000E000E000E000E0041
:106FE0000E000E000E000E0000001C001C001C0015
:106FF00000001C001C001C001C001C001C001C00CD
:107000001C001C001C001C001C001C001C001C00A0
:1070100000000000000001C001C0FFC0FFC0FFC0B1
:10702000E000E000E000E000E000E000E000E00060
:10703000E000E000E000E0000000000000000000D0
:107040000000E380E380E380E380E380E380E3808B
:10705000F780FF80FF80EB80E000E000E000E000D0
:10706000000000003FC07FC0FFC0FDC0FDC0FDC0EC
:10707000FDC0FDC07DC03DC01DC01DC01DC01DC0E8
:107080001DC01DC01DC01DC000000000000000008C
:1070900000000000000000001E001E001E001E0078
:1070A00000000000000000000000000000000000E0
:1070B000000033003300000000003F007F80FFC06D
:1070C000F3C0E1C0E1C0FFC0FFC0FF80E000E0000E
:1070D000F1C0FFC07F803F00C600C600C600C600EA
:1070E000C600E600E600F680FFC0DFC0CF40CF401C
:1070F000C740C7C0C7C0C680C600C7C0C7C0C7C0DA
:10710000000000000000000000003F007F80FFC082
:10711000F1C0E000E000FE00FE00FE00E000E00044
:10712000F1C0FFC07F803F000000000000000000B1
:10713000000000000000000000008400C600E7001E
:10714000738039C07380E700C6008400000000002F
:1071500001C001C001C0000001C001C001C001C0E8
:1071600001C001C001C001C001C001C001C071C0A7
:107170007BC07FC03F801F001E003F007F80F380E8
:10718000E000E000E000F0007E003F001F8003C050
:1071900001C000C001C0C1C0E3C0FF807F003E004D
:1071A000000000000000000000003F007F80FFC0E2
:1071B000F1C0E000F000FF007F803FC003C0C1C00D
:1071C000E3C0FFC07F803F00000000001B001B00E9
:1071D000000000000E000E000E000E000E000E005B
:1071E0000E000E000E000E000E000E000E000E002F
:1071F0000400040006000E000E000F000F00170030
:10720000170017002380238023803FC03FC041C068
:1072100041C041C0E3E0E3E0FFC0FFC038C03840F8
:1072200038403800380038003F003F8039C039C04E
:1072300038E038E038E038E038E039C0FF80FF005F
:10724000FF00FF8039C038E038E038E038E039C06E
:107250003F803F8039C039C038E038E038E038E05E
:1072600038E039C0FF80FF00FFE0FFE038603820E1
:1072700038203820382038003800380038003800EE
:10728000380038003800380038003800FE00FE00B2
:107290003FE03FE00B800B800B800B800B800B806E
:1072A0000B800B8013801380138013802380FFE0FA
:1072B000FFE0E0E0C0608020FFC0FFC038C0384081
:1072C00038403900390039003F003F0039003900AB
:1072D000390038203820382038203860FFE0FFE0BF
:1072E0006EC0E4E0E4E0D5601500150015001F0055
:1072F0001F003F803F803580358035803580358068
:1073000064C0EEE0EEE0EEE04F005F8071C041C08F
:1073100041C041C041C003800F000F0003800380C3
:1073200001C001C001C001C001C0E3803F001E00D8
:10733000FBE0FBE071C071C071C071C071C073C06F
:1073400073C077C075C07DC079C071C071C071C095
:1073500071C071C0FBE0FBE031803F801F00000086
:10736000FBE071C071C071C071C073C077C075C0DF
:107370007DC079C079C071C071C071C071C0FBE0BF
:10738000FCC0FCC0716072607260720072007400B8
:107390007C007C007E007E007E007700770073809A
:1073A00073807180F9E0F9E03FE03FE00B800B80F3
:1073B0000B800B800B800B800B800B800B800B8075
:1073C0000B800B800B80D380D380D380E7E0E7E095
:1073D000E1E0E1E061C073C073C077C077C057C01F
:1073E0005FC05DC05DC05DC05DC05DC04DC04DC0D3
:1073F0004DC049C0EBE0EBE0FBE0FBE071C071C0C9
:1074000071C071C071C071C07FC07FC071C071C0D8
:1074100071C071C071C071C071C071C0FBE0FBE090
:1074200007000F801DC038E038E0306030607070B9
:10743000707070707070707070703060306038E0B4
:1074400038E01DC00F800700FFE0FFE071C071C091
:1074500071C071C071C071C071C071C071C071C0A4
:1074600071C071C071C071C071C071C0FBE0FBE040
:10747000FF00FF8039C038E038E038E038E038E01D
:1074800039C039C03F803F0038003800380038002C
:1074900038003800FE00FE000F201FA038E07060AA
:1074A000706060206020E000E000E000E000E000AC
:1074B000E000E000E0007020702038401F800F00E6
:1074C000FFE0FFE08E208E208E200E000E000E00CA
:1074D0000E000E000E000E000E000E000E000E003C
:1074E0000E000E003F803F80F9E0F9E070C0388068
:1074F0003880388038801D801D001D001F001E0050
:107500000E000C000C00640064006C0038003000B9
:107510003F803F800E001F003F806EC06EC0CE6077
:10752000CE60CE60CE60CE60CE606EC06EC03F805A
:107530001F000E003F803F80F9E0F9E0704030808E
:107540003880390019001A000E000E000E000E00DF
:107550000B00130013802380218041C0F3E0F3E08F
:10756000FBE0FBE071C071C071C071C071C071C03F
:1075700071C071C071C071C071C071C071C071C083
:10758000FFE0FFE000600020FBE0FBE071C071C0A5
:1075900071C071C071C071C071C071C073C033C09F
:1075A0001DC001C001C001C001C001C007E007E06B
:1075B000F5E0F5E064C064C064C064C064C064C049
:1075C00064C064C064C064C064C064C064C064C09B
:1075D00064C064C0FFE0FFE07AF07AF032603260AD
:1075E000326032603260326032603260326032600B
:1075F00032603260326032607FF07FF00030001025
:10760000FF00FF00DC009C009C001C001C001C0014
:107610001F001F801DC01DC01CE01CE01CE01CE002
:107620001CE01DC07F807F00F9E0F9E070C070C0F1
:1076300070C070C070C070C078C07CC07EC07EC09A
:1076400076C076C076C076C076C07EC0FDE0F9E038
:10765000FE00FE00380038003800380038003800DE
:107660003F003F8039C039C038E038E038E038E0CA
:1076700038E039C0FF80FF008C009E00E380C1C06D
:10768000C1C080E080E000E01FE01FE000E000E01B
:1076900000E000E000E081C081C043803E001C00AB
:1076A000F380F380628066C066C066C066C06EE02C
:1076B0006EE07C606C606C606EE06EE066C066C020
:1076C00066C062806280F3800FE01FE039C071C045
:1076D00071C071C071C071C071C039C00FC007C026
:1076E00007C00DC00DC01DC019C039C071C0E3E096
:1076F0000000000000000000000000001F00638088
:107700006380738063800F80338033806380638005
:10771000638073803FC019C0004003801F803F001A
:10772000600040009F00B380E180E180E1C0E1C0E3
:10773000E1C0E1C0E1C06180738073803F001E0042
:10774000000000000000000000000000FF00738047
:107750007380738073007E007380738071C071C00A
:1077600071C071C0FF80FF00000000000000000039
:1077700000000000FFC070C070C07040700070005A
:10778000700070007000700070007000F800F80069
:107790000000000000000000000000003FC0138057
:1077A00013801380138013802380238043804380C1
:1077B000FFC0FFC0C0C0804000000000000000000B
:1077C000000000001E00330061806180E1C0FFC046
:1077D000E000E000E000E040708071803F001E00AB
:1077E0000000000000000000000000006EC0E4E0A7
:1077F000D560150015001F003F803F803580358023
:10780000358064C0EEE0EEE0000000000000000003
:10781000000000001F00338061C041C001800300F0
:107820000180018001C001C081C0C3C07F803F00D2
:10783000000000000000000000000000FBC073809A
:1078400073807380778077807B807B807B80738080
:1078500073807380FBC0FBC000000000318031806A
:107860001F000000FBC07380738073807780778077
:107870007B807B807B80738073807380FBC0FBC0C8
:10788000000000000000000000000000F8C071606F
:107890007160726072007C00770077007380738083
:1078A00071C071C0F8E0F8E00000000000000000C6
:1078B000000000001FE009C009C009C009C009C0DC
:1078C00009C009C009C0C9C0C9C0C9C073E063E02C
:1078D000000000000000000000000000E1E073C0B4
:1078E00073C073C055C055C055C05DC05DC049C0B0
:1078F00049C049C0EBE0EBE00000000000000000E0
:1079000000000000FBC073807380738073807F80F1
:10791000738073807380738073807380FBC0FBC03F
:107920000000000000000000000000003F00738025
:1079300073806180E1C0E1C0E1C0E1C0E1C061806D
:10794000738073803F001E000000000000000000F4
:1079500000000000FFC073807380738073807380A9
:10796000738073807380738073807380FBC0FBC0EF
:10797000000000000000000000000000F7007B8015
:1079800071C071C071C071C071C071C07B8077005F
:1079900070007000F800F800000000000000000017
:1079A000000000001F8033C071C061C0E000E00033
:1079B000E000E000E000E000E04070C039801F001F
:1079C0000000000000000000000000007FC04E40EA
:1079D0004E404E400E000E000E000E000E000E0037
:1079E0000E000E001F001F0000000000000000003D
:1079F00000000000F9C07080388039001D001E00B2
:107A00001E000E000C0004000800E800E8007000F2
:107A1000000000001E000E000E000E003F806EC031
:107A2000CE60CE60CE60CE60CE60CE606EC03F8055
:107A30000E000E001F001F000000000000000000EC
:107A400000000000FBC0710071003A003E001C0005
:107A50001C000E000E001F00170023802380F7C0BB
:107A60000000000000000000000000007DE039C0C0
:107A700039C039C039C039C039C039C039C039C03E
:107A80007FE07FE0006000200000000000000000B8
:107A900000000000F9E071C071C071C071C071C018
:107AA00073C03DC001C001C001C001C003E003E0DC
:107AB000000000000000000000000000EBC0C980D2
:107AC000C980C980C980C980C980C980C980C9806E
:107AD000C980C980FFC0FFC0000000000000000096
:107AE000000000007AF03260326032603260326052
:107AF00032603260326032607FF07FF00030001020
:107B0000000000000000000000000000FE00DC009B
:107B1000DC009C001C001C001F801DC01CE01CE041
:107B20001CE01CE03FC03F8000000000000000009F
:107B300000000000FDE070C070C070C070C070C078
:107B40007CC076C076C076C076C076C0FDE0F9E035
:107B5000000000000000000000000000F8007000BD
:107B600070007000700070007F00738071C071C081
:107B700071C07380FF80FF00000000000000000063
:107B8000000000003F006380C18081C001C001C0CF
:107B900007C001C001C001C001C0C18063803F00B7
:107BA000000000000000000000000000F38066C03C
:107BB00066C064606C607C606C606C606C606C6003
:107BC0006C6066C0F6C0F38000000000000000009A
:107BD000000000003FC073807380738073807380E7
:107BE0003B801F803B803B803B8073807380F7C06D
:107BF0000000000000000000000000000000000085
:107C00000000000000000000000000000000000074
:107C10000000000000000000000000000000000064
:107C20000000000000000000000000000000000054
:107C30000000000000000000000000000000000044
:107C40000000000000000000000000000000000034
:107C50000000000000000000000000000000000024
:107C60000000000000000000000000000000000014
:107C70000000000000000000000000000000000004
:107C8000000000000000000000000000C6C66C6C90
:107C900038386C6CC6C60000000000000000000010
:107CA00000000000000000000000000000000000D4
:107CB00000000000000000000000000000000000C4
:107CC00000000000000000000000000000000000B4
:107CD00000000000000000000000000000000000A4
:107CE0000000000000000000000000000000000094
:107CF0000000000000000000000000000000000084
:107D00000000000000000000000000000000000073
:107D10000000000000000000000000000000000063
:107D20000000000000000000000000000000000053
:107D30000000000000000000000000000000000043
:107D40000000000000000000000000000000000033
:107D50000000000000000000000000000000000023
:107D60000000000000000000000000000000000013
:107D70000000000000000000000000000000000003
:107D800000000000000000000000000000000000F3
:107D900000000000000000000000000000000000E3
:107DA00000000000FEFE0000FEFE0000FEFE0000DF
:107DB0000000000000000000000000000000181893
:107DC0001818181818181818180018186C6C6C6CFB
:107DD0006C000000000000000000666666FFFF66A1
:107DE0006666FFFF66666666187EFFDBD8D87C3E57
:107DF0001B1BDBFF7E1863F396F66C0C18183036ED
:107E00006F69CFC6387C6CC6C66C7C387CCDC7E643
:107E10007F3B181818181800000000000000000030
:107E20000C1C183830303030303038181C0C607072
:107E3000303818181818181838307060003C3C1882
:107E4000DBFF3C7EE700000000000000181818FF70
:107E5000FF181818000000000000000000000000DB
:107E6000001C1C1C0C180000000000FFFF0000009C
:107E70000000000000000000000000000000001CE6
:107E80001C1C030306060C0C181830306060C0C0C0
:107E90003C7E66C3C3C3C3C3C3C3C3667E3C060E76
:107EA0001E3E362606060606060606063C7EE7C386
:107EB0000303070E1C3870E0FFFF3C7EE7C3031E80
:107EC0001F030303C3E77F3E060E0E1E1E367666B3
:107ED000C6FFFF0606063F3F60607C7E6703030324
:107EE00063777E3C3E7FE3C0DCFEE7C3C3C3C3E7EA
:107EF0007E3C7F7F010307060E0C1C1838303030A3
:107F00003C7EE7C3C3E77E7EE7C3C3E7FF7E3C7EDC
:107F1000E7C3C3C3E77F3F03C3E77E3C00000038ED
:107F2000383800000038383800000000001C1C1CE5
:107F30000000001C1C1C0C180002060C183060C04D
:107F40006030180C060200000000FFFF0000FFFF79
:107F5000000000000080C06030180C060C18306073
:107F6000C0801E3F7361010103070E0C0C000C0C56
:107F70003C7EC3859DBDB5A5B7BE9CC37E3C3C7E03
:107F8000E7C3C3C3C3C3FFFFC3C3C3C3FCFEC7C3AD
:107F9000C3C6FCFEC7C3C3C7FFFE3C7EE7C3C0C069
:107FA000C0C0C0C0C3E77E3CFCFEC7C3C3C3C3C3DD
:107FB000C3C3C3C7FEFCFFFFC0C0C0C0FCFCC0C041
:107FC000C0C0FFFFFFFFC0C0C0C0FCFCC0C0C0C03D
:107FD000C0C03C7EE7C3C3C0C0C0CFCFC3E77E3CB8
:107FE000C3C3C3C3C3C3FFFFC3C3C3C3C3C318183F
:107FF0001818181818181818181818180606060649
:10800000060606060606C6C6FC78C6CECCD8D8F04C
:10801000F8D8D8CCCCCCC7C7C0C0C0C0C0C0C0C0C6
:10802000C0C0C0C0FFFFC3C3C3E7E7FFDBDBC3C300
:10803000C3C3C3C3C3C3E3E3F3F3DBDBCFCFC7C720
:10804000C3C33C7EE7C3C3C3C3C3C3C3C3E77E3C50
:10805000FEFFC3C3C3C3FFFEC0C0C0C0C0C03C7EE0
:10806000E7C3C3C3C3C3DBDFCFE77E3FFEFFC3C3AA
:10807000C3C3FFFECCCCC6C6C3C33F7FE0C0C0E0D5
:108080007C3E07030307FEFCFFFF1818181818189A
:10809000181818181818C3C3C3C3C3C3C3C3C3C3B2
:1080A000C3E77E3CC3C3C3C3C36666666666663CFD
:1080B0003C18DBDBDBDBDBDBDBDBDBFF7F3C3C3C87
:1080C000C6C6C6C66C6C38386C6CC6C6C6C6C3C3DA
:1080D000C3C3C3E77E3C181818181818FFFF03071E
:1080E000060E0C18387060E0FFFF78786060606002
:1080F0006060606060607878C0C060603030181880
:108100000C0C060603033C3C0C0C0C0C0C0C0C0C6D
:108110000C0C3C3C0C1E3361000000000000000011
:108120000000000000000000000000000000FFFF51
:108130003C1E0600000000000000000000000000DF
:1081400000387CEEC61E7EE6C6FEFF7BC0C0C0DCEB
:10815000FEE7C3C3C3C3C3E7FEDC0000003C7EE709
:10816000C0C0C0C0C0E77E3C0303033B7FE7C3C37E
:10817000C3C3C3E77F3B0000003C7EE7C3FFFFC0F3
:10818000C3E77E3C1E3E30307C7C303030303030B7
:1081900030303B7FE7C3C3C3C3E77F3B03C3FF3E2E
:1081A0006060606F7F716161616161616161181818
:1081B000000018181818181818181818181800009F
:1081C00018181818181818187870C0C0C0C0C7CE72
:1081D000DCF8F8DCCCCEC6C70C0C0C0C0C0C0C0C70
:1081E0000C0C0C0C0C0C00000066FFDBDBDBDBDB9B
:1081F000DBDBDBDB000000DEFFE3C3C3C3C3C3C3C1
:10820000C3C30000003C7EE7C3C3C3C3C3E77E3CD7
:10821000000000DCFEE7C3C3C3E7FEDCC0C0000013
:10822000003B7FE7C3C3C3E77F3B03030000003786
:108230003F3830303030303030300000003C7EE7A6
:10824000E0781E0703E77F3E303030307C7C3030F2
:10825000303030303C1C000000868686868686865C
:10826000868EFEF6000000C3C3C366666666663C83
:108270003C18000000DBDBDBDBDBDBFF7F3C3C3C56
:10828000000000C3C3E77E3C183C7EE7C3C3000088
:1082900000C3C3C3C3663C1C183870600000007F75
:1082A0007F0103071E3870607F7F060E18181818AC
:1082B0003030181818180E0618181818181818182A
:1082C0001818181818186070181818180C0C1818A6
:1082D0001818706060F29E0C0000000000000000A2
:1082E000000000000000000000000000000000008E
:1082F000FFFF6060607C7E676363636367661F7C0B
:1083000000FFFFC0C0C0C0C0C0C0C0C000000000AF
:1083100000000000001C1C1C0C180000001E78004F
:10832000FEFEC0C0C0C0C0C00000000000000000D1
:108330000039393918310000000000000000000049
:1083400000DBDBDB00000018187E7E1818181818F8
:10835000181800000018187E7E18187E7E1818184D
:108360000000003E7FE3C0FCC0FCC0E37F3E00E0B5
:10837000A1E3060C183060C0803B2A3B3C7C6C6C4F
:108380006C6C6E6F6D6D6D6DEFCE0002060C18306B
:1083900060C06030180C0602CCCCCCCCCCCCFEFF3C
:1083A000CDCDCDCDCFCEC6C6CCCCD8F8F0D8CCCCA8
:1083B000CECEC606C0C0C0C0DCFEE6C6C6C6C6C6B7
:1083C000C6C6C3C3C3C3C3C3663C1818181818185D
:1083D000003030FEFE30303E3F3333333F3E0C182A
:1083E0001C1C1C0000000000000000001C1C1C0CD9
:1083F0001800000000000000000063C6E7E7E70087
:10840000000000000000000073737331630000007F
:10841000000000000000000000183C3C18000000B4
:1084200000000000000000003C3C000000000000D4
:10843000000000000000FFFF00000000000000003E
:1084400000000000000000000000000000005B557C
:108450005151000000000000000000003C7C6C6CEA
:108460006C6C6E6F6D6DEFCE0000C06030180C0646
:108470000C183060C08000000000CCCCCCCCCCFE0E
:10848000FFCDCDCDCFCE000000C6C6CCDCF8F8DCE9
:10849000CCCCC6C60000C0C0C0C0DCFEE6C6C6C6A6
:1084A000C6C60000C3C3C3C3663C18181818181802
:1084B0000000000000000000000000000000CCCC24
:1084C000CCCCCC787830307878303030000000CCAC
:1084D000CCCCCC783030787830307CFEC6060606BE
:1084E000FEFEC6C6C6C6FE7C00004061331E1212E8
:1084F0001E33614000007CFEC6C6C6C6FEFEC6C670
:10850000C6C6FE7C18181818181800001818181875
:1085100018187EFFC3C07EFFC3C3FF7E03C3FF7E68
:108520006600FFFFC0C0C0FCFCC0C0C0FFFF000071
:108530007EFFC399A5A1A1A599C3FF7EFEFEC0C081
:10854000C0C0F8F8C0C0C0C0C0C0000000001133F7
:1085500066CC66331100000000000000000000003F
:10856000000000FFFF030000000000007E7E00000E
:1085700000000000007EFFC381B9A5BDA9A581C38D
:10858000FF7ECCCCCCCCCC78783030303030303032
:1085900000002466C3662400000000000000000004
:1085A00018187E7E1818007E7E0000007878303023
:1085B0003030303030303030FCFC001818003838A3
:1085C000181818187E7E00000000007CFEC6C6FE4B
:1085D000FEFEC6C6FE7C000000C3C3C3C3E7FFDBCC
:1085E000C3C0C0C000007FFFF3F3F37333333333F2
:1085F000333300000000001C1C00000000000000DD
:10860000006C6C007CFEC6C6FEFCC0C6FE7CCCCCFA
:10861000CCCCECEEFFFDDDDFCECCCFCF0000007E7A
:108620007E606060FCFC60606060000000000088AC
:10863000CC663366CC8800000000007CFEC60606CF
:10864000FEFEC6C6FE7CCCCCCCCCCCCCFCFCCCCCD0
:10865000CECEC6C6000000CCCCCCCCFCFCCCCCCE64
:10866000C6C6000000CCCCCCCC787830303030306E
:108670003C7EE7C3C3C3C3C3FFFFC3C3C3C3FEFE84
:10868000C0C0C0FCFEC7C3C3C3C7FEFCFCFEC7C35B
:10869000C3C6FCFEC7C3C3C7FFFEFEFEC0C0C0C04A
:1086A000C0C0C0C0C0C0C0C01E3E766666666666FA
:1086B0006666FFFFC3C3FEFEC0C0C0C0FCFCC0C0F6
:1086C000C0C0FFFFDBDBDBDBDBDB7E7EDBDBDBDBA2
:1086D000DBDB3E7F6303031E1E07030303677F3E4E
:1086E000C3C3C3C3C3C7CFDFFBF3E3C3C3C3667E48
:1086F00000C3C3C3C7CFDFFBF3E3C3C3C6CECCD82D
:10870000D8F0F8D8D8CCCCCCC7C70F1F3B33333305
:1087100033333333333373E3C3C3C3E7E7FFDBDB05
:10872000C3C3C3C3C3C3C3C3C3C3C3FFFFC3C3C3A1
:10873000C3C3C3C33C7EE7C3C3C3C3C3C3C3C3E78D
:108740007E3CFFFFC3C3C3C3C3C3C3C3C3C3C3C34D
:10875000FEFFC3C3C3C3FFFEC0C0C0C0C0C03C7ED9
:10876000E7C3C0C0C0C0C0C0C3E77E3CFFFF18184D
:1087700018181818181818181818C3C3C3C3C3C377
:10878000663C18181838F0E018187EFFDBDBDBDBDE
:10879000DBDBFF7E1818C6C6C6C66C6C38386C6C3E
:1087A000C6C6C6C6C6C6C6C6C6C6C6C6C6C6C6FE31
:1087B000FF03C6C6C6C6C6C6FE7E06060606060673
:1087C000DBDBDBDBDBDBDBDBDBDBDBDBFFFFDBDBB1
:1087D000DBDBDBDBDBDBDBDBDBFFFF03F0F03030A5
:1087E00030303E3F333333333F3EC3C3C3C3C3C3D1
:1087F000F3FBDBDBDBDBFBF3C0C0C0C0C0C0FCFEB7
:10880000C6C6C6C6FEFC3C7EE7C303031F1F0303A8
:10881000C3E77E3CCEDFDBDBDBDBFBFBDBDBDBDB79
:10882000DFCE1F3F736363733F1F1B333373E3C399
:10883000000000387CEEC61E7EE6C6FEFF7B003FD1
:108840007FE0C0DCFEE7C3C3C3E77E3C000000FE60
:10885000FFC3C3FEFEC7C3C3FFFE000000FEFEC091
:10886000C0C0C0C0C0C0C0C00000003E7E6666661A
:10887000666666FFFFC30000003C7EE7C3FFFFC0E3
:10888000C3E77E3C000000DBDBDBDB7E7EDBDBDB8B
:10889000DBDB0000003E7F63030E0E0303677F3EB9
:1088A000000000C3C3C3C7CFDFFBF3E3C3C3667ECF
:1088B00000C3C3C3C7CFDFFBF3E3C3C3000000C6DD
:1088C000CECCD8D8F0F8DCCCC6C70000000F1F3BD8
:1088D00033333333333373E3000000C3C3E7E7FFBD
:1088E000DBDBC3C3C3C3000000C3C3C3C3FFFFC3F9
:1088F000C3C3C3C30000003C7EE7C3C3C3C3C3E715
:108900007E3C000000FFFFC3C3C3C3C3C3C3C3C3D4
:10891000000000DCFEE7C3C3C3E7FEDCC0C000000C
:10892000003C7EE7C3C0C0C0C3E77E3C000000FF40
:10893000FF181818181818181818000000C3C3C317
:10894000C3663C1C183870600018187EFFDBDBDB48
:10895000DBDBFF7E1818000000C3C3E77E3C183C39
:108960007EE7C3C3000000C6C6C6C6C6C6C6C6FEEE
:10897000FF03000000C6C6C6C6FE7E060606060643
:10898000000000DBDBDBDBDBDBDBDBDBFFFF000036
:1089900000DBDBDBDBDBDBDBDBFFFF03000000F00E
:1089A000F030303E3F3333333F3E000000C3C3C39B
:1089B000C3F3FBDBCBDBFBF3000000C0C0C0C0FC9B
:1089C000FEC6C6C6FEFC0000003C7EE7C31F1F03B8
:1089D00003E77E3C000000CEDFDBDBDBFBFBDBDB09
:1089E000DFCE0000001F3F7363733F1F333373E319
:1089F0004A616E000000000000000000000000005E
:108A00000000000046656200000000000000000059
:108A100000000000000000004D6172000000000036
:108A20000000000000000000000000004170720023
:108A30000000000000000000000000000000000036
:108A40004D617900000000000000000000000000FF
:108A5000000000004A756E000000000000000000E9
:108A600000000000000000004A756C0000000000DB
:108A700000000000000000000000000041756700D9
:108A800000000000000000000000000000000000E6
:108A900053657000000000000000000000000000AE
:108AA000000000004F6374000000000000000000A0
:108AB00000000000000000004E6F76000000000083
:108AC000000000000000000000000000446563009A
:108AD0000000000000000000000000000000000096
:108AE000D8D2D0C8D52DCC2D3032D4002530326428
:108AF0002E253032642E25303464003E64000000A0
:108B00000000021FC800001CC8000019C8000015A2
:108B1000C8000012C8000015C8000019C800001CD9
:108B2000C800001FC800000000000219BC020019A4
:108B3000B0040119BC020019B0040119BC020019EB
:108B4000B0040119BC020019B0040119BC020019DB
:108B5000B0040119BC020019B0040119BC020019CB
:108B6000B0040119BC020019B0040119BC020000D4
:108B70000000024003A001CF006700330022001074
:108B80000088134C0EB90B240A0D093F089E071DDF
:108B900007B20658060A06C6058B05560556055641
:108BA00005560556055605560556055605560556ED
:108BB00005560556055605560556055605560556DD
:108BC00005000032006400C8001B222B37445365A7
:108BD0007A91AAC6E3FAFE00030C0F30333C3FC083
:108BE000C3CCCFF0F3FCFF30313233343536373875
:108BF000394142434445460030313233343536370B
:108C0000383961626364656600286E756C6C20702B
:108C10006F696E74657229003F3F3F0000014F5F2E
:108C200000495F0045165F0002085F00117A5E0090
:108C30000B3C5E0001975E0001165F0001145F00AF
:108C400001085F0002975E00052B5E00016E5E006A
:108C5000017A5E0003445E00027A5E0003775E00E4
:108C6000FB00C60000007E2000000000760000002F
:108C7000082000F6C4008A927A926A925A924A9226
:108C8000BA93AA939A938A93FA93EA933A922A927E
:108C90001A920A927A936A93E4D14FB658B669B69B
:108CA0007BB68CB600E008BF0093CB480093CC485D
:108CB0000091D748002379F00A9579F00A9579F068
:108CC0000A9579F00A95A9F00A95C1F00A95C1F0C4
:108CD0000A95C9F01FC047D10EC045D104C031D19B
:108CE00001C03DD138D102E02DD100E40093A506AA
:108CF00011C035D130D102E025D109C030D101C039
:108D000020D129D101C02FD102E00093250600E433
:108D10000093A6060E946652002309F4D9C0009170
:108D2000D7480395083009F400E00093D74842E0A3
:108D30000E945D48442309F0DAC00E943F55202F6D
:108D4000212B09F4C5C02091E148222319F430E019
:108D50003093D920013230E010408CF00091D920BE
:108D6000002369F481E89BE8F0D0059114912F313C
:108D7000B8014AE050E090F4DDD023950BC081E8C3
:108D80009BE8222349F001E00093D920DED0CCD02B
:108D9000D1D02A95208304C0FC01C6D00E9475481A
:108DA0006093DD487093DE480093DB481093DC4805
:108DB0000091DD481091DE480093260910932709A1
:108DC000E6D001E00093460600000000E1D03093B9
:108DD000400930936009309361093093460930931C
:108DE0004709EFEBFBE8A591B491B595A7950091E4
:108DF000E1480A3060F412E0019FE1E8FBE8E00D91
:108E0000F11D059114918BD08AD0A00FB11FAA0F2C
:108E1000BB1FE3ECFBE805911491A00FB11F9897DD
:108E200000E089EC9BE84091EB205091EC20FC01A4
:108E300024912417350770F4053010F41A9706C0F2
:108E4000083010F4989702C0A055B04003950196E1
:108E50000E3068F3A0936809B0936909009168091E
:108E600010916909000F111F00936609109367099B
:108E700001E00093D82048E450E025ED39E8609106
:108E8000D3897091D48909E4709F702D609F710D12
:108E9000200D371F08E810E20E9475600E94FC5305
:108EA00004E00093400900E10093460603E085D00A
:108EB000E1EDF9E830E03BBF028113810F5F1F4F06
:108EC000028313830039114091F4328333830FC03E
:108ED00000E000930009009320090093210900930A
:108EE00006090CE00093250601E00093F0488CBED3
:108EF0007BBE69BE58BE4FBEADD0699179910990D5
:108F0000199029903990E991F99189919991A991B4
:108F1000B9914990599069907990899018951595D3
:108F20000795159507950895659174914AE050E06D
:108F30008B0108950E947548E1EEF8E43BBF208163
:108F4000089501E000932606089502E0209F800D19
:108F5000911DFC01089504E00093A606089501E028
:108F600000932506089501E00093260604E000938F
:108F7000A506089527D000E10BD0000000000000F6
:108F80000000000000E20093460611D0189500E3AF
:108F900000934506089516D0FADF00E000934009DB
:108FA000009360090093610908D001D0189528BF8B
:108FB0001FBF0991199129910895009346090093C3
:108FC0004709089578942A931A930A931FB728B7EC
:108FD00000E008BF08957894FA93EA9342D02FB73F
:108FE00048B75BB700E008BF7894009121020050B9
:108FF00069F0085091F00852A9F427D00093E720B7
:109000001093E82000E01CD00BBF10C01ED00093CE
:10901000E9201093EA2008E006C017D00093EB2067
:109020001093EC2000E30CD030E03BBF00810068DF
:1090300000835BBF48BF2FBF0DD0E991F991189510
:1090400000932102E0E2F2E00895009124021091E1
:1090500025020895099119912991399149915991C0
:1090600008955A934A933A932A931A930A93089528
:109070000C947A62FF24F8BE03E40DBF04E20EBF35
:10908000C4E4D1E3E0E0EABF0E94DD4E002311F02A
:109090000E94CC600E9433540E9447600C94384870
:1090A0000024E8E0001FEA952AF0001C0416D0F323
:1090B000041AF8CF402D00950895FF27442312F499
:1090C000F1604195002312F4F09501950E945048FB
:1090D000F0FD0195F1FD41950895149F102D059F18
:1090E000100D049F002D110D089500241124E0E1BE
:1090F000101104C0E850102F0FEF0894001F111F2B
:10910000EA9542F0001C111C04161506B8F3041A67
:10911000150AF4CFA001009510950895FF27552357
:1091200012F4F1600FD0112312F4F09507D00E94D1
:109130007548F0FD03D0F1FD05C008951195019526
:109140001040089551954195504008952224349F30
:10915000302D259F300D169F300D079F300D249F19
:10916000202D310D159F200D311D069F200D311D25
:10917000149F102D210D321D059F100D211D321D34
:10918000049F002D110D221D321D089544FF03C0C0
:10919000980110E000E043FF04C0322F212F102F70
:1091A00000E0477031F0000F111F221F331F4A9556
:1091B000D1F7089544FF03C0890130E020E043FF68
:1091C00004C0012F122F232F30E0477031F0369565
:1091D0002795179507954A95D1F7089500241124EE
:1091E0001001E0E22015300571F4E051312F202FFD
:1091F0001FEF0FEF0894301106C0E850322F212FD7
:10920000102F0FEF0894001F111F221F331FEA9524
:1092100072F0001C111C221C331C041615062606B5
:10922000370688F3041A150A260A370AECCFA0017C
:10923000B1010095109520953095089530952095B1
:10924000109501951F4F2F4F3F4F0895FF27172E61
:10925000660F771F089409F4771F6795EE27032E92
:10926000220F331F089409F4331F279508952223F2
:1092700042F0323030F03A95EE0F001F111F221FDE
:10928000C2F7E03821F400FF08940EF488940F4FE1
:109290001F4F2F4F3F4F323038F4332319F427FD3F
:1092A00031E002C027FF30E03F3F29F0220F000CE1
:1092B00037952795089589C0032E002012F40E9447
:1092C0001E49E02F012F122F232F3EE9E894CFCF24
:1092D000F901EE0FFF1F37FBFF3F31F0EF2BE12BC2
:1092E000E02B8894B8940895EE2321F00894989484
:1092F000B89408959894889438940895FB01EE0FDB
:10930000FF1F77FBFF3F31F0EF2BE52BE42B889419
:10931000B8940895EE2371F3E9CFF0DF68F021F4FB
:109320003723262F8A010895372FFBCFE7DF20F060
:109330000BF008957327EAF74CC0CADFE8F3B3F3E4
:1093400061F3DCDFC8F383F3A1F380DF401751073B
:109350006207730729F4302C3124E2F400242FC073
:1093600058F0F9019B01BF01F8018A01AF01E0E06B
:10937000F0E0302C012C132C731B39F066955795B7
:109380004795F795E0407395C9F7E7FBEE0FE0E0EE
:1093900010246AF0EF0F041F151F261F60F4279595
:1093A00017950795E79508F46894339560CFEF0B10
:1093B000040B150B260B5BCFE0E87E27BECF302DCC
:1093C000307822271127002708953FE7302920E829
:1093D000F9CF3FEF2FEFF6CF91DFD8F3D1F37078CD
:1093E000372708958BDFA8F3A3F3F9CF3078372719
:1093F00098CF6EDF70F383F3A9F380DF50F3B3F3FC
:10940000A9F324DF0124E8943F57E040370FEF1F12
:1094100012F021F0DACF3A3E90F26894302C049F9B
:10942000F001059F7727F00D711D149F2224F00D88
:10943000711D221C069F0027700D211C001F249FF8
:109440004427700D211C041F159F700D211C041F43
:10945000169F1127200C011D111F259F200C011D97
:10946000141F269F000D111D5EF433951695079568
:1094700027947795F795E79533953130BCF314C071
:10948000112322F0332349F433950EC0339561F450
:10949000032C9BCF3A95313038F0EE0FFF1F771F2A
:1094A000221C001F111FB2F7E894FE2B09F06894EC
:1094B000212F102F022DE72F032CE3CE09DF48F0D8
:1094C00039F01CDF30F00417150726073707089519
:1094D00015CF989408951894089510DFA0F0F8DE41
:1094E00090F029F0E32FE7273AF47317089506DF89
:1094F00051F04EF008940895041715072607370712
:1095000019F016F4B8F788940895F8DEE0F3E0DE79
:10951000D0F3E7DFC0F308940895F0DE20F01BF0ED
:1095200070783727089555CFE9DEE9F3E0F3032E8D
:10953000072645CF032E072648CFCADEA0F36BF3DC
:1095400099F3DCDE80F39BF3A9F380DE012427FD91
:1095500006C03150E040000F111F221FD2F767FDF7
:1095600006C07150F040440F551F661FD2F7E894B3
:10957000371BEF0B3158EF4F2AF0EE23E9F63F3F50
:10958000D9F203C0393EA8F26894E0E0F0E0401759
:109590005107620738F0315008F46894000F111F2A
:1095A000221FEE1F71E01124222409C0000F111F99
:1095B000221FEE1F041715072607EF0720F0041BD4
:1095C000150B260BEF0B771F111C221C78F7000FD1
:1095D000111F221FEE1F041715072607EF073E2E47
:1095E000F0F9E894E0E839F008F4E0E0322A312AB2
:1095F000302A09F06894709510942094332311F068
:10960000F0FF09C0269417947795E79508F46894BD
:1096100033953130BCF3072F112D222D32CE1EDEB3
:109620003F5748F03F3168F007FCC9CE3FE72FEFC6
:109630001FEF0FEF089530E020E0890110E000E017
:109640000895432F322F212F102F0E2F4F51419568
:109650000E94DA4807FE08950C941E49479117901E
:1096600011FA2790379007900CBE0895F7DF041B7E
:1096700010E000C020E030E000C028F110FC25C060
:1096800047910790E00FF11F0417100540E02407F1
:109690003407C8F486F412FE05C0E00FF11F0791ED
:1096A000069002C006910024F101E01BF0090CB7FE
:1096B00000400CBF1994E00FF11FE00FF11F27903D
:1096C000379007900CBEF101199411F4C6F7E3CF5F
:1096D000319612FC31960EF0329650E060E070E068
:1096E00047914B3F48F079F34F3F29F04E3F11F03F
:1096F0007791679157914791041B150B260B370BF8
:1097000029F308F3E5CFAF93BF93D8013BBF29BF3F
:1097100001900D92415050406040D1F7BF91AF9100
:109720000895FA92EA92DA92CA92BA92AA929A9218
:109730008A927A926A925A924A92BA93AA939A9386
:109740008A930895FF84EE84DD84CC84BB84AA844C
:10975000998488847F806E805D804C80BB81AA81E3
:1097600099818881F0E0EC0FFD1FEF0108950FEF64
:1097700000937E2000937F20089520917F203091D8
:109780007E200AD020937E2030937F200895009180
:109790007E2010917F2008952027022F02950F70C0
:1097A0002027022F122F110F110F110F110F312728
:1097B00040E2049F202531250895392F482F202F7E
:1097C000212B21F0C80107D00197E9F7842F932FAF
:1097D000089501D000C000000000089544D0006842
:1097E0000083089538D004D000810F7B0083089552
:1097F00000810F7700830081006400830895BA938D
:10980000AA939A93D801132E26D0208711863287E7
:10981000648775873687452B0B81402B0C81402B45
:1098200042830D811E810483158339BF20814985C0
:10983000442311F000E201C000E02C7D5F81252B64
:10984000202B2C93442311F0088506839991A9912C
:10985000B99127960895F80130E03BBF089503D0F1
:10986000046000830895F7DF00810895F4DF238307
:109870000895F9DF00610083089528D00DD0B9D094
:1098800001FFFDCF008100FDA1601DD0B9F7D9D047
:10989000B0D001FFFDCF20C0B3D0AA0FD5C016D0E5
:1098A000FBDFA7D001FFFDCF008100FDA1600BD041
:1098B000B9F705D0C8D093D001FFFDCF0DC001E0AE
:1098C00000938106089558D1BA950895BA938DD022
:1098D000C801A0E0B8E008954FD101E0B6D0FC0186
:1098E000A08330D2A991B99108953BD17BD0229722
:1098F000DA95098369017A01BB2402C001E02AD10B
:1099000043D1098126D1002309F050C00E94B74BF2
:109910001CD188811AD11881912F082F012B09F4AD
:1099200045C0813001E0100708F040C0F60130E08A
:109930003BBF808311834FD0A8800A2D08D1882493
:1099400099242E0102E0400E581CDC01119721C021
:10995000662408E0702E54D0660C76D04AD001FF01
:10996000FDCF008100FF02C0689460F805D17A94B1
:1099700091F7A5DF68D033D001FFFDCFFDD02DD00A
:109980006882F20161922F01E1D001E0800E00E0D7
:10999000901E8A169B06E0F21ED0A8818E016DDF14
:1099A000B8810E94C74BA017B10741F0F1D0B39422
:1099B0000AE0B01608F4A2CF02E309C0AC019E0190
:1099C0002E5F3F4F87010E947560E2D00A2D2296DC
:1099D000D39506D1AFC08E0162CF01E036C00E94A0
:1099E000E94B08C05A924A92BA93AA939A938A93DF
:1099F000089506D0E8E8F6E030E03BBF0081089526
:109A00000C94EB4BF3DF902F88E097FB01E016F40A
:109A10001CD001C055DF990F16D0B2D001FFFDCF89
:109A2000ABD08A9591F70DD0E4DF01FFFDCF008127
:109A300000FF02C000E301C000E012E010938106C5
:109A400081C101E002D0DCDF02E0009382060895CC
:109A500088D05A924A92C9DFF02EE12EA22F6A01D5
:109A60009924832E29010FEF400E501E02C00AE0F8
:109A700071D08AD00F2D71D009F04FC00E94B74B22
:109A80000A2F65D00A2F69D009F047C0082D5FD092
:109A9000082D63D009F041C00E2D59D00E2D5DD098
:109AA000E1F566247724C60108C0AA2465D0AA205F
:109AB000A1F501E0600E731E01966414750408F5AB
:109AC000FC0130E03BBFA0800A2D41D0BA2C08E059
:109AD000A02EB7FA01E016F4B8DF01C0F1DEBB0C2E
:109AE000B2DF4ED001FFFDCF47D0AA9491F7A9DF96
:109AF00080DF01FFFDCF008100FFD7CF00E3A02E64
:109B0000D5CF0E94C74B912FA02E21D00A2D21D056
:109B1000092F1DD0092F1DD0A02E3AD0AA2029F040
:109B2000939405E0901608F4A2CF0A2D0BD1A991C9
:109B3000499059906990799089909990A990B9909D
:109B4000C990D990E990F990089545DF08810C9467
:109B5000BD4B58CF10E00C94125054DFA02E0023C0
:109B60000895FA92EA92DA92CA92BA92AA929A92D4
:109B70008A927A926A92089502E00093810608958B
:109B80003FDF00918806089505E02ED008D02FC051
:109B900006D001D001E00093820605E025C001E077
:109BA00026D002E008951EDF812F2B0112E0019FD5
:109BB000A8E0B0E2A00DB11D182F90E099BF0C9164
:109BC00047DF002351F409E10FD04E815F819201FC
:109BD000182FFD019BBF018188DE02D022960895D7
:109BE00080DE49905990089510E00C94DD4B00936D
:109BF000810605E010E00C94DD4BF8DEEF97EF975F
:109C0000679700910621002309F499C000E00093B2
:109C10000621EAEDF0E230E00BBF068917890A83DE
:109C20001B8300A511A50C831D830091080607FF67
:109C300003C001E0088701C038870E943F550E83AA
:109C40001F830E945A5509871A87009107210A9598
:109C500019F00A9589F023C07CD04C5F5F4F2AE051
:109C600030E011E000E09FDF002309F068C00C85C0
:109C700007FF17C001E016C0CE01845A9F4F8C0128
:109C800020E0E9E0F1E230E049E350E060E00E94EA
:109C9000834B5FD0425A5F4F2AE312E0E3CF55D0A7
:109CA0004EC000E0009308210D8500FF04C000E2D3
:109CB0000093A50603C000E20093A6060D8501FFF0
:109CC00004C000E10093A50603C000E10093A606CE
:109CD0000E85013009F439D00E85023019F403E005
:109CE0001BE835D00E85033019F40BE21BE82FD0AA
:109CF0000C850F70053039F40F85073020F40E9471
:109D0000AC590E9411520C85007F41F0AE01455FB5
:109D10005F4F21E530E001E00E9481550B85002373
:109D200059F000E0EAEDF0E20BBF02A703A701E063
:109D300004A70B8505A703C001E000930721EF9658
:109D4000EF9667968991999108950BEF1AE80C9414
:109D500003538E01055F1F4F1A930A93BE016E5F76
:109D60007F4FAE0108950BEC0093520008E0009382
:109D7000500008ED04BF03E00093410008EC00939D
:109D80005500E1E5F0E0FBBF008103FFFCCFE0E51B
:109D9000008100610083E1E5008104FFFDCF08ED53
:109DA00004BF04E00093400008950093400400E2E3
:109DB000009361060093660608952AD104E000939B
:109DC000C5070093C1070FEF0093E4060093E00678
:109DD00000932007C8DF01E0E8DF00915D04087F01
:109DE000036000935D0400E000935E0400935F0451
:109DF00000915C0400780D6200935C0400000895FB
:109E000044D10FE4009324060093210604E000935C
:109E1000C4070CE00093C007FBD007E70093A1063E
:109E200003E0009382060093860607E00093000893
:109E300008E311E000932608109327081093060802
:109E400007E00093A200AAEDB0E20EED10E0FD01E4
:109E50001BBF0587168705EC0787108B07E000936B
:109E6000040201E00093200200930202009300022A
:109E700004E00093010201E00093220200E300935A
:109E80002102E0E2F2E0008100680083E093A50691
:109E900000E10093A50605E0FD01068B178BA4D019
:109EA0000E945B60012B11F091E001C090E091D025
:109EB00040815181628173814132534465467748C4
:109EC00019F04424439401C04424042D0170192F37
:109ED0001170012BB9F140FACEF40E943E530023D9
:109EE000A9F47CD088D0F1F700E10093A60684EFB6
:109EF00091E081D0F1F772D07ED0F1F700E10093CC
:109F0000A60680ED97E077D0F1F7EBCF81E04FE246
:109F10002AD18D010E949B604092DE209093E02028
:109F200009E00093DA208093FD205ED00E947560E6
:109F300041E253E465E677E84CD040835183628385
:109F4000738301C080E000E00093E12001E0009312
:109F5000DD200093012100E00093F22010E0FD01DC
:109F6000018F028F02A703A706A702E005A71187AA
:109F7000082F0E9445540E94725501E00E94E7524A
:109F800044E0F1D00DEC19E80E949B600E94115250
:109F900000EA0093810600E80093850600E2009342
:109FA000860602E00093B60A00EC0093B50A08E1C9
:109FB0000093B40AE0E0F1E0EBBF008100680083A9
:109FC0000E940154789489919991A991B9914990ED
:109FD0000895ECEFFFEF30E03BBF089500E1009300
:109FE000A50684EF91E0089548E050E020E230E2D9
:109FF00000E010E208950197E6EBF5E00091001112
:10A00000002309F0A8953197C9F7082F092B089567
:10A0100003E3009344060093410608950E94DF5035
:10A020000C94BD50392F482F202F212B61F0015067
:10A03000104086EB95E020910011222309F0A895AD
:10A04000019791F3F8CF842F932F08955A921DD042
:10A0500080E090E000EF402E09E8502E03E010E091
:10A06000F20130E0ACE0B0E20E944661012B41F029
:10A07000019604E1400E00E0501E8C30900770F312
:10A0800001968C01A0DF599008954A92BA93AA9341
:10A090009A938A93089553D06496089564974CD008
:10A0A00005D058D06496089505D00FC098012F5F51
:10A0B0003F4F0895649720E230E202D00C942C6167
:10A0C0004FD02AE330E08E0108950C1B1D0BFE01DA
:10A0D000E00FF11F30E03BBF30834AE050E020E06A
:10A0E0003CD0649608955A924A929A938A9327D0C4
:10A0F000C801ACDF280120D00F5F1F4F98012AD084
:10A10000000F111F000F111F0429152920E20FD085
:10A11000082A002D192B0BD0802D912FC5DF082B7D
:10A12000192B649689919991499059900895129F9D
:10A13000102D029F1129089508D00C946061649736
:10A1400004D00E942C61B2DF05C020E230E00CE0B8
:10A1500010E2089505D04AE006D08E010C94776293
:10A160008E010C943A6150E020E030E008950CD26A
:10A1700009C10CE00093250608950091680604FDCE
:10A180000BC061D006FD12C017D004FD0FC00FD068
:10A190000065068B178B089556D006FF07C00CD0BC
:10A1A00004FF04C004D00F7A068B178B0895EAEDE4
:10A1B000F0E206891789089550D0E8E649C0009179
:10A1C000C8072091F0203091F12001FB16F4346093
:10A1D00001C03B7F2093F0203093F120089500913F
:10A1E000080603FD0AC02FD002FD10C02FD003FDCA
:10A1F0000DC025D00460068B089525D002FF06C04F
:10A2000025D003FF03C01BD00B7F068B0895009160
:10A21000080604FD0AC017D000FD10C017D004FDC9
:10A220000DC00DD00160068B08950DD000FF06C053
:10A230000DD004FF03C003D00E7F068B0895EAED16
:10A24000F0E2068908950091F020089506D0E8E034
:10A25000F6E030E03BBF0081089501E010E00C948F
:10A26000125001E0A4D102E083C102E0A0D101E0DC
:10A270007FC10091064000230895009128060895AB
:10A280008395EBDF853008958A93002351F10A9579
:10A29000F1F501E00093E62063D0E3DF80E0EDDF3D
:10A2A00004FF03C0EDDF20F401C080E0E2DFB9F776
:10A2B00060D0E3DF04FD05C0E3DF20F0DADF39F52D
:10A2C00003C080E0D6DFA9F746D071D101E000934A
:10A2D000E320EAEDF0E2A2D000A5016000A7899199
:10A2E000089500E00093E62001E03AD0BEDF80E070
:10A2F000C4DF04FF28C0C4DF38F1BBDF29F339D045
:10A30000BCDF04FD24C0BCDF18F1B3DFE9F223D0C9
:10A310002FD105E010E02FD103E049D108E512E08C
:10A320002AD1E0E0F0E47AD00481158103331307E9
:10A330003CF02EE1129F102D029F002D110D1BD11C
:10A3400003E016D1CCCF80E094DF91F6BDCF80E062
:10A3500090DFB1F6B9CF00E00093064003E0089526
:10A360000093064000E0E0E0F0E40BBF04830583C7
:10A37000089500E00BD1F7DF80E008951093CB48FB
:10A380001093CC480CE0F0D01093E1480895E8E039
:10A39000F6E044D0008107FF32C0ECE5F0E4008134
:10A3A00003950083043021F410915A40112321F0C9
:10A3B00010915B40011781F5308300915A400023D2
:10A3C00019F00AE000935B4001E000935A40E8E096
:10A3D000F6E0008107FF0CC001E0E0916F40F0E083
:10A3E000E15AFF4B0083EFE6F0E400810395008320
:10A3F00000916F40003181F430936F4008950091D7
:10A400005A40002349F030935A4000E500935B40E6
:10A4100030935C4030935E400895FC0130E03BBFD8
:10A4200008954FD09A938A9389E091E20AEF0093BE
:10A43000122104E110E0E0EEFAE830E0DC011A96C7
:10A440000E94896000E0009327210E947350E5DF9D
:10A45000078F10A30E944E5028010E942650D80159
:10A460000E944B502ED01A930A934CEE5AE860E0AB
:10A470000AE211E20E940E61269600917740009355
:10A48000342101E00093352100E412E0C6DF05A786
:10A4900016A702EE14E007A710AB00E911E001AB2C
:10A4A00012AB08EC03AB34AB04E605AB36AB06E409
:10A4B00007AB30AF89919991A991B9914990599081
:10A4C00008955A924A92BA93AA930895BCDE0474EE
:10A4D000043011F000E0089501E008958A9310E03F
:10A4E0004DDF1093D74888E013C00091D748002370
:10A4F00079F00A9579F00A9579F00A9581F00A9534
:10A5000091F00A95A1F00A95A1F00A95C1F01DC03D
:10A5100047D00AC045D004C033D02FD00DC03BD0A7
:10A5200002E02BD010C037D002E01ED004C033D0E0
:10A5300007C026D01FDE1BD004E016D006C030D0E6
:10A5400002E018DE14D004E015DE0091D748039530
:10A55000083009F400E00093D74805E00CD014D08F
:10A560008A9519F68991089500932606089500E4C6
:10A570000093A60608950C941250F6DF00E417C06D
:10A5800011D0F6DF02E0089500E010E00093CB4820
:10A590000093CC48089501E00093250604E0E8CF3D
:10A5A00001D005C001E00093260604E00895009361
:10A5B000A50608954DE123D009E510E40E949B60B3
:10A5C00000E500935B4000E000935A40089510E4DA
:10A5D00010932506002319F04CE70DD007C044E086
:10A5E0000AD032D142E50BD007E010E42DD1E2DFF2
:10A5F00006E00C94AC5903D000E010E4089550E05C
:10A6000020E030E00895BA93AA93F80100910A403F
:10A61000023031F100E510E030E0A7E0B0E40E9444
:10A62000896001E00093584000E00093574006E045
:10A630000093400800E000936008009361080091D7
:10A64000574014E0019FF001E050F04C30E03BBF78
:10A650000781009366083093670801E0009346087D
:10A66000A991B991089500E400932606089500E0A9
:10A670000093024000E4009325060895BA92AA923E
:10A680009A928A927A926A925A924A92BA93AA9328
:10A690009A938A9384D008E7802E06E5902E04E3EF
:10A6A000A02E02E1B02E80E082D09DD0B0F4482FE1
:10A6B000840195010E94C6486BD00E94DA4861D09F
:10A6C0008395803209F480E08D01292F30E0082540
:10A6D00019252A253B2575D0E8CF67D084D018F5F9
:10A6E00099BF0D911D912D913C9166D0AD01692FBF
:10A6F00070E0482559256A257B250417150726078C
:10A70000370769F5A4505AD08A958F3F09F48FE135
:10A71000482F840195010E94DA483AD00E94C64829
:10A7200030D058D0DBCF3BD042D05DD030F400E009
:10A7300010E020E030E045D0F8CF37D054D098F486
:10A74000FD01392F932FDF01A45038D03BBF40814A
:10A75000518162817381452B462B472B11F000E01C
:10A7600003C038D0EBCF01E089919991A991B991BB
:10A77000499059906990799089909990A990B99051
:10A78000089542015301802A912AA22AB32A0895EA
:10A790002801390140E2481B84019501089500E039
:10A7A00010E420E0D801922F0895A45007D000248F
:10A7B000112422243324089599B7A350B040904027
:10A7C000089599BF0D931D932D933C93F5DFAC5FD6
:10A7D000BF4F9F4F01E0000E00E0101E00E0201E62
:10A7E00000E0301E089500E0001600EF100601E0C2
:10A7F000200600E03006089529D000E50CD00C9426
:10A80000394C48E5FCDE00E810E21ED01FD008E518
:10A8100002D00C94394C10E01A930A931A931A93AD
:10A8200060EB7AE050E140E020E830E200E111E046
:10A830000E94FF4B06D00E942F4C2FE802D00E94AE
:10A84000364C00E111E008950C949B60FADF0E9401
:10A85000F24BF7DF0E94EE4B00E00A9301E00A930F
:10A8600000E00A9308950E94004F00E20093A506BD
:10A8700000E10093A6060E940E500E9406590E9415
:10A880005A540E94FD4DA895F6CF002341F041E6B1
:10A8900050E020E030E000E918E40E949B600E9454
:10A8A0006E5200E00093E2480093E34801E0009319
:10A8B000F04808958A93EA970E946652002319F49B
:10A8C0000E9472555CC000910821002309F173D0E9
:10A8D00056C077D001EF18E4000D131FF8018AD09D
:10A8E0002681322F3F7049F03A9589F13A9599F1D6
:10A8F0003A9599F13A95D1F103C054D00E94465847
:10A900006AD055D011F00E94A75504E00093C60705
:10A910000E945A55012B99F104E00093C507A895B0
:10A9200050D0E1EFF8E4E00DF31F64D084814AE3F6
:10A9300050E034969F018E010E9475608A9511F057
:10A940008A95F1F61FD00F3511401CF218C02AD09D
:10A950000E94CE55D5CF2FD0D3CF29D081F012D0A1
:10A96000012B79F611D00E94C65808C020D039F0CA
:10A9700009D0012B31F608D00E94E6582CD0EA9677
:10A98000899108950C943F550AEF18E44091F348DB
:10A990005091F44823E5529F502D429F510D000DD8
:10A9A000151F089522952F70075F1F4F089500917E
:10A9B000F0480023089504E00093C5070093C607FC
:10A9C00008952091F3483091F44803E5309F302DED
:10A9D000209F310D0895E1EFF8E40CD0028113813E
:10A9E0000F5F1F4F02831383083C104011F4328322
:10A9F0003383089530E03BBF0895AA939A938A93D6
:10AA0000A22F202F212BB9F1C80148E450E020E00B
:10AA100030E005ED19E82090D1893090D28969E4C1
:10AA2000369E302C269E310C000D131D0E949B601B
:10AA30004091D1895091D28909E4509F502D409F77
:10AA4000510DE02DF52FE35EF547D4DFA083F89498
:10AA5000E1EDF9E8008111810F5F1F4F0083118341
:10AA6000019700810039114011F4308331837894CB
:10AA7000082F092B51F689919991A991089500E029
:10AA800010E0F894D8D10BBF42815381608171816D
:10AA90004617570769F08B01461757071CF4041B2C
:10AAA000150B06C000E911E0041B150B060F171F5C
:10AAB0007894089547D04281538100811181041711
:10AAC000150719F400E010E00895401751071CF431
:10AAD000041B150B089508EC041B350B4081040F73
:10AAE000131F08954CED50E420E030E001EF18E42E
:10AAF00048D244E152E720E030E001ED19E80C943F
:10AB00009B60202EB9018A0179D323E530E0529F62
:10AB1000502D429F510DE02DF52F75D33BBF248260
:10AB2000AB01980106EF18E42090F1483090F2480C
:10AB300063E514D307D023D3083C104011F43083CD
:10AB400031830895E1EFF8E430E03BBF089500E081
:10AB50000093F04800930009009320090093210915
:10AB6000009306090093E1480093E5480093E64806
:10AB70000E94B7500AE010E00E94125004E00093D7
:10AB8000000900E00093060908E813E10093260994
:10AB90001093270902E0009306090895AA928A9269
:10ABA0007A92D4D2EF972D97D801722E19D3818142
:10ABB0008280438000E1400E662447FA1EF4E89448
:10ABC00047F86394A480B7D20C5F1F4FDAD108E432
:10ABD000A01608F0AA2470E0092F10E00A0D171F34
:10ABE0000834104014F098E49A19AAD20C5F1F4F51
:10ABF0000A0D9ED2042D015109F4A2C00A9581F0DC
:10AC00000A9509F48DC00A9509F44EC00A9509F415
:10AC1000A3C00A9509F4E8C00A9509F4F4C004C178
:10AC2000A5D200EF11E064E1662011F051E001C00F
:10AC300052E05A9578D229E430E0329E302C229EA0
:10AC4000310CAAD1F31D30D14CE090E037D138E27D
:10AC5000739F72D1239532D16AD115D17CD14A9597
:10AC6000A9F71DD1408128E2429F66D10294202D90
:10AC7000FFD02881FDD029812295FED0FD012083BF
:10AC8000DAD08081918101968083918380399140CF
:10AC900019F420E020832183552359F60E5F1F4FBE
:10ACA0006A9509F4BEC0C0CF8FD1E6D175D1F31F2C
:10ACB00000D19AD2708220E06CE08201000F111F57
:10ACC00080EF91E0800F911F5ED1FC0121D15BD11B
:10ACD000800D911DFC01D7D090E03DD16A9581F7A0
:10ACE000DBD028E2629FE0EFF1E023D1E00FF11F1B
:10ACF00005911491088319830295AFD00881ADD0D6
:10AD000009810295AED0FD0100830DD1A1D009F0DB
:10AD10000AD168D108F085C096D008F082C0C5CFAE
:10AD200053D168D140FB0EF4FFD023D211F49083AD
:10AD300091834F5F5F4F4E30590708F072C0F1CFDB
:10AD400043D158D185D009F0EED04CD108F069C07C
:10AD50007AD008F066C0F5CF09D200EF1BE75EE0BD
:10AD60006091D1897091D28929E434D215D1F71F2D
:10AD70009BD04FE090E01ED199BF6D938DD0639F23
:10AD8000D7D064912395362F3695369599BF3D934C
:10AD900095D03EE0CCD07491239530E4639F372F5B
:10ADA00032953F70032A99BF0D9204D17295707F3E
:10ADB00034E0639F712999BF7D93660F660F99BF39
:10ADC0006D934A95C1F637D0608171816F5F7F4F77
:10ADD000608371836039714011F4908391830F5FB8
:10ADE0001F4F5A95F1F0BCCFDAD0EBD00201000C26
:10ADF000111C60EF7BE265D0C9F7A4D0EBD088F4DA
:10AE00001DD078F4F2CFCBD0DCD00201000C111CA5
:10AE100060EF73E556D0C9F795D0DCD010F40ED0B2
:10AE200098F3272D082DC3D0EF962D9674D17990E5
:10AE30008990A9900895E1EDF9E808954F5F5F4F7B
:10AE40004431530708954F5F5F4F443159070895C8
:10AE5000042F0170162D1023089503D099BF0D9370
:10AE600008950F70E02FF0E0E952F447049108953F
:10AE700003D099BF2D9308952F70E22FF0E0E9528F
:10AE8000F44724910895059014900A821B8223951B
:10AE9000888182958F70089502D060810895FE01A7
:10AEA0003496E20FF91F089504D03BBF708220E072
:10AEB0000895DF011496E45BFF4F0895F0DF708181
:10AEC0000895600D711D29D018E2019EFB0120D06C
:10AED00024D0019E600D711DFB01659174916A8300
:10AEE0007B832395188139BF1D936A817981707F97
:10AEF000162F12951F70712B39BF7D936295607F5D
:10AF00001B8112951F70612B39BF6D930A950895AF
:10AF1000E00DF11D12D023950895FE013496E20F45
:10AF2000F31F0080089501E0400E591E0895739F9D
:10AF3000F801E00DF11D0895FBDF059014900882E3
:10AF40001982089501E0400E531E82DF19F001E0DE
:10AF5000400E531E08950ED088810BD0898108D0F1
:10AF60008A81E82FE295EF70FF2705D002D08B8110
:10AF700082958F70FC01E952F447349199BF3D935B
:10AF800008950C949B60FE01349630E0E20FF31FAD
:10AF9000708138E2739F08954EDFE00D08954424D8
:10AFA000552403D040E050E00895272D082F10E0ED
:10AFB0000C94FD5471DF3EE0639FBADF64912395EA
:10AFC00008954FD008E10895F0DF4424552440E06F
:10AFD00050E00895CED011F43083318304E140165F
:10AFE00053060895C6D011F49083918304E140166E
:10AFF0005906089536D068E18201000F111F90E0D4
:10B000005DDF32E022D008821982239557DF1DD000
:10B010000A821B822395788199BF7D937A818981E9
:10B02000807F372F32953F70832B99BF8D93729518
:10B03000707F8B8182958F70782B99BF7D936A95F5
:10B04000F9F601E0400E591E0895739FF001E0519A
:10B05000F64D05901490000E111EF001059014900D
:10B0600008950AD0E1EDF9E8E00DF31F22DF30E0AA
:10B070003BBF708220E008952091D1893091D28920
:10B0800009E4309F302D209F310D08958A925ED0C3
:10B09000EF972997D801622EA3D0418052808381F7
:10B0A000848049D06EDF08E4801608F0882470E0C0
:10B0B000092F10E0080D171F0934104014F098E410
:10B0C00098193ED0080D34D0262D042D70DF48E4A9
:10B0D00050E09E0105ED19E826D069E43FD040918B
:10B0E000D1895091D28909E482D0E35EF5477CD0C2
:10B0F0006082F8943ED011F4308331837894082F25
:10B100008A95002321F7262D052D51DFEF962996EC
:10B1100002D08990089589919991A991B991499006
:10B120005990699008952090D1893090D2890895DE
:10B13000151F0C94756048E450E020E08E010895DE
:10B14000492F50E015969D018E0108956A925A92FA
:10B150004A92BA93AA939A938A930895369E302C72
:10B16000269E310C000D131D0C947560272D082FA1
:10B170001ECFE1EDF9E803D00039114008950081B8
:10B1800011810F5F1F4F008311830895BA93AA9313
:10B19000D801E0E0F0E400E00BBF008309BF0D91AF
:10B1A00001830C9103830023A8ECB7E00C9139F0E4
:10B1B00001FF07C00E943753A991B991089501FF7B
:10B1C000F9CF01E002830E943353F6CF0CD0008107
:10B1D0000C94445130E0729F702D629F710D089560
:10B1E00090E099BF9C91F80130E03BBF0895509FDB
:10B1F000502D409F510DE02DF52F08954091F148BD
:10B200005091F2480895EF50F74B0895BA93AA93DE
:10B210009A938A932297D85000918E48002309F47C
:10B2200094C000E000938E4892D10023F1F0DE013B
:10B23000AE5FBB4F102FE0918448F0918548EC57EA
:10B24000FF4B82D1208190E039BF2D93E4E8F8E4F0
:10B25000408151814F5F5F4F408351834030544064
:10B2600011F4908391831A9531F79E012E5F3F4F21
:10B270003A932A93BE016E5F7F4FAE014C5F5B4FE6
:10B28000802F90E001969C0113E001E00E94D34DD5
:10B29000002309F05AC0888199818230904008F4D7
:10B2A0004DC050D1008105FFFCCFF89400E07BD168
:10B2B00062D139F060D11CF4241B022F02C0041BA0
:10B2C000020F78947894002361F79981863090403A
:10B2D00018F001E000938F4820E088819981019760
:10B2E00030E010C0FE013296E20FF31F0081E091C2
:10B2F0008A48F0918B48EC57FB4B0083EAE8F8E46E
:10B30000DFD023952817390768F3F8940DD1008111
:10B31000E1EAF8E0108115FFFDCFCED0789401E08E
:10B320000683088119810230104079F408EE13E099
:10B330000E94DD4B01E00093062107C000918F4879
:10B34000002319F000E000938F482296D85F89917E
:10B350009991A991B99108959A938A9318E01093BD
:10B3600045061093410612E0019FE3E7FBE8E00D7C
:10B37000F11D259131972093A608259124912093C2
:10B38000A70813E01093A50814E11093A30818E18F
:10B390001093A408009377401CD000E000938448E9
:10B3A0000093854800938648009387480093884817
:10B3B0000093894800938A4800938B4800938C48F7
:10B3C00000938D4800938E4800938F4889919991FE
:10B3D00008958091784090917940863900E09007F7
:10B3E00034F44AE050E08C010E948E483CC08A3F11
:10B3F0009007B4F485593CD0392F46E950E060E01D
:10B4000070E0349F202D010C302D149F102D210D44
:10B41000351F049F002D110D251F351F4AE021C047
:10B42000895F26D0292F392F48E95AE360E070E080
:10B43000349F302D259F300D249F202D310D159FD9
:10B44000200D311D149F102D210D361F059F100D4D
:10B45000211D361F049F002D110D261F361F4AE0A7
:10B4600050E00E94EE4800937A4010937B4008958C
:10B4700090408C01990F990B0895FA93EA935BD051
:10B480002FB748B75BB700E008BF0091A0085AD0BB
:10B49000108114FD0AC0E0918648F0918748EC576E
:10B4A000FF4B0083E6E8F8E40BD05BBF48BF2FBF3B
:10B4B00034D0E991F99118950093A008E8E8F8E4F0
:10B4C000008111810F5F1F4F0083118300301440F2
:10B4D00011F4308331830895FA93EA930A927A93B0
:10B4E0006A9329D06FB778B70BB600E008BF46D093
:10B4F000012B49F019D028D00081E1EAF8E0108151
:10B5000015FFFDCFD9DF0BBE78BF6FBF06D06991A5
:10B5100079910990E991F9911895099119912991D9
:10B520003991499159910895E0918848F09189485D
:10B53000EC57FB4B08955A934A933A932A931A93E4
:10B540000A930895E1EAF8E030E03BBF089500E097
:10B5500010E020918648309187484091844850916E
:10B56000854809D039F007D024F48901041B150B54
:10B57000089513D0089542175307089510E013D08B
:10B580004217530741F04217530724F48901041B63
:10B59000150B01C002D07894089514E0041B150B1C
:10B5A000020F131F0895F89420918A4830918B4818
:10B5B000409188485091894808956A925A924A92D7
:10B5C000BA93AA939A938A93FA93EA933A922A9215
:10B5D0001A920A927A936A9303D1AFB7B8B749B671
:10B5E0005BB66CB600E008BF78940E94C75100912A
:10B5F00002400023C9F0E8D0008103950083009148
:10B60000034000230091C80719F001FD0BC002C0E0
:10B6100001FF08C000910040043620F41091014061
:10B62000011710F00E94375300910640002351F09B
:10B63000CBD00481158176D004831583073910405F
:10B640000CF03683E0E9F8E4C1D003AD14AD6AD064
:10B6500003AF14AFE091CB48F091CC483B9714F086
:10B660000E94B9500E94EF500E940751EAEDF0E2AB
:10B67000ADD0018D128D56D0018F128F80917C40FC
:10B6800090917D400196813707E190074CF080E072
:10B6900090E0ECE7F0E40281138144D0028313834D
:10B6A00080937C4090937D40EAEDF0E202A513A5E3
:10B6B00039D002A713A7E0910421F0910521329718
:10B6C0003CF0309304213093052101E000930621E2
:10B6D000ECE8F8E40081118125D000831183E0912A
:10B6E0008C48F0918D4832973CF030938C483093E1
:10B6F0008D4801E000938E486CBE5BBE49BEB8BF6A
:10B70000AFBF67D0699179910990199029903990CC
:10B71000E991F99189919991A991B991499059909B
:10B72000699018950F5F1F4F0895FA93EA931A9244
:10B730000A9256D02FB748B75BB700E008BF78949D
:10B740000091574014E0019FF001E050F04C3ED0D2
:10B7500000851185015010400087118700915740E6
:10B760002CD000851185012B39F002850023E1F4EE
:10B7700002E00093470618C0E7E5F0E40081039576
:10B7800000831BD00285023051F402E0009345068D
:10B7900030934008309346083093584005C00781E5
:10B7A00000936608309367085BBF48BF2FBF11D076
:10B7B00009901990E991F991189514E0019FE0E042
:10B7C000F0E4E00DF11D0895E0E0F0E430E03BBF6F
:10B7D00008950991199129913991499159910895A3
:10B7E0005A934A933A932A931A930A9308950E947C
:10B7F000914B3CD45A016B017B018824992459D187
:10B800005ED128F1A2D30E945E4AD9F509890023AE
:10B8100009F448C08A149B044CF40CEF80160FEF17
:10B82000900624F000E0088BA818B9080FEFA00ECE
:10B83000B01E0A890023A1F100E0098B33C031D189
:10B840000E949D4A13D40AE0800E00E0901E47EB50
:10B8500053E46AEB71E532D190F340E050E060E2EE
:10B8600071E42CD198F60E949D4A00D401E0800E2C
:10B8700000E0901EF2CF15D1F7D306EF800E0FEF48
:10B88000901E40E057EE6BED7EE210D1A0F311D197
:10B890000DD108F0BBCF60E271E4E6D3D9D3F7CF86
:10B8A00001E00A8B0889002319F06624772455C02B
:10B8B00099203AF500E3F2D0B5010A2D0B2919F4CD
:10B8C0000A89002311F00EE2E5D06624772406C031
:10B8D00000E3F701DFD00FEFA00EB01EBDD386143A
:10B8E00097041CF40A2D0B2999F70FEF1FEF061B85
:10B8F000170B801691060CF47AC0772466246394A3
:10B900002CC034017194619400E0700A26C0D9D033
:10B910000E940F4B402E212F220F220B322F0E940C
:10B920005C49A801B901CDD00E94DC49A801B90148
:10B9300000E010E020E231E497D3042D005DAED0AA
:10B94000930101E058D3232B41F40A2D0B2919F45C
:10B950000A89002311F00EE2A2D0A614B704BCF6A7
:10B9600040E050E060EA70E4A9D008F040C061E037
:10B97000F70131974BBF00810E3249F0060F00836B
:10B980000A3321F400E3008361E001C060E08F012D
:10B990003197C016D10670F360FB4EF5088900237D
:10B9A000B1F0F70102C000833197CE16DF0658F4DC
:10B9B000DF0149BF0E910E32B1F7DF0112970C91F2
:10B9C00000833197F1CF01E0800E941E0DC001E09D
:10B9D000E00EF41EF70105C0DF0149BF0E910083A0
:10B9E0003197CE16DF06C0F301E3F6010083098923
:10B9F000002321F40DC00FEFE00EF01EF70111D36C
:10BA000002910033C1F30E3219F40FEFE00EF01E75
:10BA100008890023A1F1F70104D30193992032F49E
:10BA20000DE238D091948194930A02C00BE232D097
:10BA30008CD20AE0E00EF31E6F5F7F4F45D0405D71
:10BA4000F7013BBF41937F013FD04801012BA1F794
:10BA5000623073078CF33B018B0115D03BBF208113
:10BA6000830111D0E60FF71F3B9720836150704090
:10BA7000613073078CF706EFE00E0FEFF01E8701C1
:10BA8000E3E10C94A24B119501951040F701E00FF2
:10BA9000F11F08953BBF01937F010895F701C1D2C3
:10BAA000FACF49EF52E065E170E508950AD00C94B1
:10BAB0006D4A40E050E060E87FE3089502D00C94C6
:10BAC000854A8C019D0108954AE050E084010C9460
:10BAD0008E480E94914BEF97EF976E975BD24D8700
:10BAE0005E876F8700E00A870B878FD2E255FF4F92
:10BAF000E080F18005C06ED251D205E241D25BD226
:10BB000000E0088B098B0A8B03C048D239D253D28C
:10BB100080D2053249F00023C1F70A851B85EF96D4
:10BB2000EF966E96E4E1ADCFEA81FB815CD20532FF
:10BB300011F300E0098708870F8309833E0106E1BE
:10BB40005AD207EE1BE817D205C01981112309F458
:10BB5000098340D245D2102F1052B9F3135059F037
:10BB60001850B1F3125019F0135049F00CC00F8166
:10BB700003950F83EECF088503950887EACF0985E3
:10BB800003950987E6CF0A32A9F4F7012BBF56D2F5
:10BB9000A80158D253D20D831E8311234AF40D817C
:10BBA0001195019510400D831E830F8103950F831E
:10BBB000ECD110C02D832E834AE050E009C00D81E6
:10BBC0001E81D0D1020F151F005310400D831E831C
:10BBD0000DD2A8F30F81002311F000E0098700D2F5
:10BBE0000E32D9F4F7D1E02FFB8106910A3229F405
:10BBF00028D240805180C9D113C0442455244AE042
:10BC000050E0F4D168F48201ADD12801420E551EF6
:10BC100000ED400E0FEF501EF4CF44244A94542CF4
:10BC200080E0EA811B812C81F12F2BBF06910C54FF
:10BC300021F00C5119F0045031F481E0EF5F1F4FF7
:10BC4000EA831B832C83E5D10883ECE1F0E0FBBFA2
:10BC5000FCE80C94364BECD14E5F5F4F4083518330
:10BC60004A855B853EF4652F660F660BACD1628317
:10BC7000638346CFA8D144CFE4D100810E8B6E01FF
:10BC800007E1C00ED31E16C1DCD160807180062D85
:10BC9000072939F409E01CE8088B198B3A8B0DE071
:10BCA00007C1552022F400E1402E07E2502E8824DF
:10BCB000992403C001E0800E931EF3013BBF019164
:10BCC0003F01002319F084149504A4F3C5D1630146
:10BCD00091948194930A680C791CECC00885002328
:10BCE00031F0042D052919F455244424439408EF18
:10BCF0001BE841D10881003739F4A3D12ED100E1EE
:10BD0000802E00E0098331C093D136F432D1808196
:10BD10009181A281B38102C095D11FD108810F36D4
:10BD200011F408E0EDCF053751F70AE0E9CF80D1F3
:10BD300036F41FD1408151816281738107C082D165
:10BD400040815181652F660F660B762FCA01DB019A
:10BD500077234AF40DE209839095A095B0958195DB
:10BD60009F4FAF4FBF4F0AE0802E3E010BE943D1FA
:10BD70006E010BE9C00E00E0D01E082F092B0A2B24
:10BD80000B2B19F001E00C8705C000E00C87042D97
:10BD90000529C1F064D10B891C893D89000D111D55
:10BDA000F80121D140D15BD161D1012B022B032BB2
:10BDB00089F755203AF40985002321F05AD102C0B1
:10BDC00000E331D18E0105561F4FC2D0CCF3088558
:10BDD000002309F46FC00C8500FF6CC00881083790
:10BDE00011F0083549F438D108811AD1008334D1D3
:10BDF00000E3F30100835EC00F3609F05BC010D191
:10BE00000081003309F456C000E302933F0152C0A1
:10BE100088248394088102500883042D052939F46D
:10BE200055244424439408C000E008838824552006
:10BE30001AF406E0402E5524FCD09BD0FFD022817E
:10BE4000338140E081D00E946D4A18F44DE249836D
:10BE50003058AE014A5E5F4F6D817E81660E571F7E
:10BE6000752E48854A938A924A814A93662D752F8A
:10BE7000A201BDDC680109850023E1F0FAD030E0C1
:10BE8000860166D0BCF400E3F3013BBF02933F019F
:10BE9000F7CF0A811B812C81015010407BD008E133
:10BEA0001CE820E0088B198B2A8B6624772403E09A
:10BEB000C02EDD242601461857080D811E81041569
:10BEC00015051CF48824992408C0DAD08D808418C4
:10BED0001509912E10E0801A910A0F81002331F488
:10BEE00003C08DD000E262D0B3D0DAF7098100231D
:10BEF00059F085D008C0E455FF4F4081518190D062
:10BF000001913F01352F52D00FEF400E501E82F0AD
:10BF1000088919892A89012B022B77D061F370D007
:10BF2000E889F12F2BBF0791E88BF98B2A8BEBCF98
:10BF30000F81002309F4E4CD8BD00AF4E1CD2ED09B
:10BF400000E2422F33D0F8CF50E060E070E0089577
:10BF50000619170904151505089580819181A0E03F
:10BF6000B0E008950E946D482791EA83FB833C83EB
:10BF700008954C5F68C020E00B8B1C8B2D8B0895BF
:10BF8000ED85FE856F856CBF08950A811B812C812C
:10BF90000F5F1F4F0A831B832C830895DE019AB71E
:10BFA00099BFA455BF4F2D913C910895ED85FE8515
:10BFB0002F852CBF242F19950A851B850F5F1F4FD6
:10BFC0000A871B870895F8010081F181E02F4083E3
:10BFD000518308958F010F5F1F4F0A831B83C7CFC3
:10BFE000EA81FB813C813BBF0691089515D0069103
:10BFF00000530A300895600E00E0701E089505D0C9
:10C00000E455FF4F408131810895FE013AB73BBFAF
:10C01000089502D00791A9CFEA81FB813C81F7CF37
:10C02000F30130E0F4CFF301FCDF02933F01089508
:10C0300080FBF701F6DF02D0A8010895008111818D
:10C040000895F7DF4E5F5F4F40835183F8010895F5
:10C050000FEF800E901E08950FEF600ECECF31DDF2
:10C06000482D72DF0C94EE480E94F949C801D901AD
:10C07000089506D04D805E8010E0401A510A089560
:10C080000981002311F001E0089500E008950C9467
:10C090003848F80103C0319641505040042F052B19
:10C0A00039F030E03BBF00810217A9F78F010895F6
:10C0B00000E010E00895BD01F801D90102C041502F
:10C0C0005040042F052B69F030E03BBF019139BF90
:10C0D0001D910117A1F318F40FEF1FEF04C001E049
:10C0E00001C000E010E0DB0108950C01CA01B801B5
:10C0F000A90130E009C0FA013BBF2191AF01FB016A
:10C100003BBF2193BF010197282F292BA1F7C00125
:10C110000895792FAD01202F212B51F03BBF27919E
:10C1200090E099BF2D9301501040202F212BB1F7A3
:10C130008A01972F0895BC01CA01F80104C030E0BC
:10C140003BBF21930197382F392BC9F7CB010895B5
:10C1500040E099BF4D9399B70150104020403040C6
:10C16000402F412B422B432B99F70895232F8F010A
:10C17000F8012BBF07902BB78F01FD019BBF0192E8
:10C180009BB7DF014150504060407040342F352B49
:10C19000362B372B69F7089502E6402E0CE8502E17
:10C1A00000E0602EF201362D6BBE479157916791EA
:10C1B0007691F201EC5FFF4F3F4F3BBFA791B791E4
:10C1C0009691F201362DE95FFF4F3F4F3BBF07913C
:10C1D00017913691F801012B032B11F0C7DF03C033
:10C1E0008A019B01B5DF0AE0400E00E0501E601E90
:10C1F00006E71CE820E040165106620698F2089512
:10C20000602FF90130E03BBF00811181A8014F5F31
:10C210005F4F40835183F8016083089524970A8318
:10C220001B838A01262FAE014C5F5F4F48835983E1
:10C23000AE015A934A93AE014C5F5F4F5A934A93B3
:10C2400040E051E660E00E94695D20E0EA81FB8108
:10C250002BBF208324960895F80130E03BBF008176
:10C26000021731F031960023C1F700E010E0089585
:10C270008F010895AD01F901D80130E03BBF219154
:10C2800039BF2D932223D1F7DA010895592F02C027
:10C2900001501040202F212B79F090E099BF2D9173
:10C2A0003BBF4791241731F018F40FEF1FEF06C082
:10C2B00001E003C0222361F700E010E0952F08950C
:10C2C000F80100E010E030E03BBF4081421709F484
:10C2D0008F0131964423C1F708950E94914B2C970A
:10C2E0000E831F832C833D836A837B833A010A81FB
:10C2F0001B81012B31F040E0EA81F12F4BBF4083DD
:10C3000041834E805F8030E001C0EDD0F2013BBF41
:10C31000008190E0802F099785309040B0F3003283
:10C32000A1F30D3211F00B3219F431962F0101C037
:10C330000BE2098355230AF46BC001E06016530732
:10C3400009F466C005E2601653070CF061C001E015
:10C35000601653075CF000E160165040C9F4BFD08E
:10C36000B9F401810062083799F40BC0B8D011F01C
:10C370000AE00CC001810062083739F400E1602E48
:10C38000772402E0400E531E03C008E0602E77249D
:10C39000720101C0A8D0A3D0E9F380E090E0A0E052
:10C3A000B0E06201A72CAA0CAA0819C08887998757
:10C3B000AA87BB87202F29552883AC01BD018301A3
:10C3C0002A2D3A2D0E94A648A801B901088130E023
:10C3D000400F531F631F731FCA01DB0184D0F2019A
:10C3E0003BBF408150E0FA01E154F0407A9710F0F1
:10C3F000242F03C0405E5F4F9A01A30109E510E2BC
:10C400000E944960202F212B89F6E414F50489F459
:10C410000C811D81012B41F04E815F81EC81F12F58
:10C4200030E03BBF4083518300E010E020E030E08B
:10C4300052C0A2014C195D09F301EC5CFF4D30E0E4
:10C440003BBF0081401B504092F141305040D4F43A
:10C4500048818C019D01041B104020403040801712
:10C460009107A207B30770F0A3016A2D7A2D0E94ED
:10C47000EE48088419842A843B840015110522059E
:10C480003305A9F002E210E000934221109343210A
:10C490000A811B81012B31F041E050E0EA81F12F4C
:10C4A000408351838FEF9FEFAFEFBFEF0AC0098149
:10C4B0000D3239F49095A095B09581959F4FAF4F6F
:10C4C000BF4F0C811D81012B21F0EC81F12F4082A7
:10C4D00051828C019D012C96E0E10C94A24BF2015B
:10C4E00000810033089501E0400E531E089560E07E
:10C4F00070E0F3CEFFCFF4F5FCFD4F6374203236CD
:10C5000020323031360000000000000000003230E0
:10C510003A35323A343800000000000000000000D4
:10C52000000000002115110E0D0C0B0B0A0A090961
:10C53000090909080808080808080707070707077E
:10C5400007070707070707303132333435363738E6
:10C55000396162636465666768696A6B6C6D6E6F8A
:0CC56000707172737475767778797A00C8
:0400000300009074F5
:00000001FF
